:100000000C94D1110C94F9110C94F9110C94F91170
:100010000C94F9110C94F9110C94F9110C94F91138
:100020000C94F9110C94F9110C94F9110C94F91128
:100030000C94F9110C94F9110C94F9110C94F91118
:100040000C94FC290C94F9110C94CA290C94A42941
:100050000C94F9110C94F9110C94F9110C94F911F8
:100060000C94462A0C94F91100000000230026008D
:10007000290000000000003E5B4F5B3E3E6B4F6B73
:100080003E1C3E7C3E1C183C7E3C181C577D571C79
:100090001C5E7F5E1C00183C1800FFE7C3E7FF00F2
:1000A00018241800FFE7DBE7FF30483A060E262940
:1000B000792926407F050507407F05253F5A3CE703
:1000C0003C5A7F3E1C1C08081C1C3E7F14227F22C9
:1000D000145F5F005F5F06097F017F006689956A94
:1000E000606060606094A2FFA29408047E0408101F
:1000F000207E201008082A1C08081C2A08081E1048
:100100001010100C1E0C1E0C30383E3830060E3EFF
:100110000E06000000000000005F0000000700075E
:1001200000147F147F14242A7F2A12231308646288
:1001300036495620500008070300001C22410000E9
:1001400041221C002A1C7F1C2A08083E0808008047
:1001500070300008080808080000606000201008DF
:1001600004023E5149453E00427F400072494949E0
:10017000462141494D331814127F10274545453912
:100180003C4A494931412111090736494949364616
:100190004949291E000014000000403400000008F6
:1001A0001422411414141414004122140802015999
:1001B00009063E415D594E7C1211127C7F49494926
:1001C000363E414141227F4141413E7F49494941BB
:1001D0007F090909013E414151737F0808087F00EA
:1001E000417F41002040413F017F081422417F4070
:1001F0004040407F021C027F7F0408107F3E414147
:10020000413E7F090909063E4151215E7F091929B6
:1002100046264949493203017F01033F4040403FA0
:100220001F2040201F3F4038403F631408146303E1
:10023000047804036159494D43007F414141020460
:10024000081020004141417F040201020440404067
:100250004040000307080020545478407F2844445D
:10026000383844444428384444287F385454541877
:1002700000087E090218A4A49C787F080404780072
:10028000447D40002040403D007F10284400004154
:100290007F40007C047804787C0804047838444467
:1002A0004438FC1824241818242418FC7C0804045E
:1002B00008485454542404043F44243C4040207CC7
:1002C0001C2040201C3C4030403C44281028444C1A
:1002D0009090907C4464544C4400083641000000E7
:1002E000770000004136080002010204023C262388
:1002F000263C1EA1A161123A4040207A3854545540
:100300005921555579412254547842215554784009
:1003100020545579400C1E52721239555555593991
:100320005454545939555454580000457C410002E6
:10033000457D420001457C407D1211127DF028254B
:1003400028F07C545545002054547C547C0A097F85
:100350004932494949323A4444443A324A48483099
:100360003A4141217A3A42402078009DA0A07D3D4B
:100370004242423D3D4040403D3C24FF2424487ED3
:100380004943662B2FFC2F2BFF0929F620C0887EBE
:10039000090320545479410000447D413048484AC3
:1003A00032384040227A007A0A0A727D0D19317D76
:1003B0002629292F28262929292630484D4020384A
:1003C0000808080808080808382F10C8ACBA2F1009
:1003D0002834FA00007B000008142A142222142A70
:1003E00014085500550055AA55AA55AAFF55FF55A2
:1003F000FF000000FF00101010FF00141414FF0095
:100400001010FF00FF1010F010F0141414FC001472
:1004100014F700FF0000FF00FF1414F404FC141490
:1004200017101F10101F101F1414141F001010108D
:10043000F0000000001F101010101F10101010F01E
:1004400010000000FF101010101010101010FF10FE
:10045000000000FF140000FF00FF00001F10170045
:1004600000FC04F414141710171414F404F400001E
:10047000FF00F714141414141414F700F7141414D0
:10048000171410101F101F141414F4141010F0106F
:10049000F000001F101F0000001F14000000FC14DB
:1004A0000000F010F01010FF10FF141414FF1410CF
:1004B00010101F00000000F010FFFFFFFFFFF0F022
:1004C000F0F0F0FFFFFF0000000000FFFF0F0F0F34
:1004D0000F0F3844443844FC4A4A4A347E0202062C
:1004E00006027E027E0263554941633844443C045F
:1004F000407E201E2006027E020299A5E7A5991CD7
:100500002A492A1C4C7201724C304A4D4D303048F9
:10051000784830BC625A463D3E494949007E010157
:10052000017E2A2A2A2A2A44445F444440514A44EC
:100530004040444A51400000FF0103E080FF0000BA
:1005400008086B6B083612362436060F090F0600B2
:100550000018180000001010003040FF0101001FBB
:1005600001011E00191D1712003C3C3C3C0000001C
:10057000000000000000240027002A000000000006
:10058000250028002B0004040404040404040202CF
:100590000202020203030303030301020408102002
:1005A000408001020408102001020408102000000D
:1005B0000008000201000003040700000000000022
:1005C0000000FFFFFFFFFFFFFFFFFFFFFFFFFFFF39
:1005D000FFFFFFFFFFFFFFFFFFFFFFFFFFFFFFFF2B
:1005E000FFFFFFFFFFFFFFFFFFFFFFFFFFFFFFFF1B
:1005F000FFFFFFFFFFFFFFFFFFFFFFFFFFFFFFFF0B
:10060000FFFFFFFFFFFFFFFFE3FFFFFFFFFFFFFF16
:10061000FFFFFFFFFFFFFFFFFFFFFFFFFFFFFFFFEA
:10062000FFF0FFFFFF1FFFFF00000000FFFFFFFFC5
:10063000FFFFFFFFFFFFFFFFFFFFFC7FFFFF1FFF2D
:10064000FF00000000FFFFFFFFFFFFFFFFFFFFFFB6
:10065000FFFCFFFF3FFFFF1FFFFC000000003FFF0C
:10066000FFFFFFFFFFFFFFFFFFFFF87FC7BFFFFF99
:100670001FFFFC7FFFFFFE3FFFFFFFFFFFFFFFFFAE
:10068000FFFFFFF83FE39FFF8F1FFFFC7FFFFFFE91
:100690003FFFFFFFFFFFFFFFFFFFFFFFF01FF99F7F
:1006A000FF8F1FFFFC7FFFFFFE0FFFFFFFFFFFFF1E
:1006B000FFFFFFFFFFF00FB9DFFF8F1FFFFC7FFF82
:1006C000FFFE07FFFFFFFFFFFFFFFFFFFFFFF0073A
:1006D0009DFFFF8F1FFFFC7FFFFFFE07FFFFFFFF58
:1006E000FFFFFFFFFFFFFFF0031FFFE38F1FFFFC74
:1006F0007FFFFFFE07FFFFFFFFFFFFFFFFFFFFFF83
:10070000F0007FFFE38F1FFFFC7FFFFFFE07FFFF6F
:10071000FFFFFFFFFFFFFFFFFFF000FFFFE38F1F63
:10072000FFFC7FFFFFFE07FFFFFFFFFFFFFFFFFF55
:10073000FFFFF800FFFFE38F1FFFFC7FFFFFFE07B7
:10074000FFFFFFFFFFFFFFFFFFFFFFF8007FF8E362
:100750008F1FFFFC7FFFFFFE07FFFFFFFFFFFFFF75
:10076000FFFFFFFFFC003FF8E38F1FFFFC7FFFFF51
:10077000FE07FFFFFFFFFFFFFFFFFFFFFFFC001F64
:10078000F8E38F1FFFFC7FFFFFFE07FFFFFFFFFF68
:10079000FFFFFFFFFFFFFE000FF8E38F1FFFFC7F4F
:1007A000FFFFFE07FFFFFFFFFFFFFFFFFFFFFFFF52
:1007B0000007F8E38F1FFFFC7FFFFFFE0FFFFFFF27
:1007C000FFFFFFFFFFFFFFFFFF0003F8E38F1FFFA7
:1007D000FC7FFFFFFE3FFFFFFFFFFFFFFFFFFFFF6D
:1007E000FFFF0001F8E38F1FFFFC7FFFFFFE3FFCD0
:1007F00003FFFFFFFFFFFFFFFFFFFE700638E38FE1
:100800001FFFFC000000003FFC03FFFFFFFFFFE7AE
:10081000FFFFFFF83FFE38E38F1FFFFF00000000DF
:10082000FFFF9FFFFFFFFFFFE7FFFFFFF01FFE3807
:10083000E38F1FFFFF00000000FFFF9FFFFFFFFF90
:10084000FFE7FFFFFFE00FFFFFFFFFFFFFFFFFFFDF
:10085000FFFFFFFF9E0C07060A78C126983FFFFFA7
:10086000FFFFFFFFFFFFFFFFFFFFFFFFFF9E7C93E8
:10087000227832672609FFFFFFFFFFFFFFFFFFFF20
:10088000FFFFFFFFFFFF9E7C93327926672649FF1B
:10089000FFFFFFFFFFFFFFFC0000000000007F9E46
:1008A0001C933219E66726787F8000000000000F55
:1008B000FC0000000000007F9E7C933279E06726F8
:1008C00079FF8000000000000FFC00000000000025
:1008D0007F9E7C932679E6672679FF8000000000E2
:1008E000000FFC0000000000007F9E0C930609E64C
:1008F000618E783F8000000000000FFFFFFFFFFFC8
:10090000FFFFFFFFFFFF3FFFFFFFFFFFFFFFFFFFB7
:10091000FFFFFFFFFFFFFFFFFFFFFFFFFFFFFF3FA7
:10092000FFFFFFFFFFFFFFFFFFFFFFFFFFFFFFFFD7
:10093000FFFFFFFFFFFFFFFF3FFFFFFFFFFFFFFF87
:10094000FFFFFFFFFFFFFFFFFFFFFFFFFFFFFFFFB7
:10095000FF3FFFFFFFFFFFFFFFFFFFFFFFFFFFFF67
:10096000FFFFFFFFFFFFFFFFFFFFFFFFFFFFFFFF97
:10097000FFFFFFC3FFFFFFFFFFFFFFFFFFFFFFFFC3
:10098000FFFFFFFFFFFFFFFFFFFFFFFF81FFFFFFF5
:10099000FFFFFFFFFFFFFFFFFFFFFFFFFFFFFFFF67
:1009A000FFFFFFFFFF18FFFFFFFFFFFFFFFFFFFF3E
:1009B000FFFFFFFFFFFFFFFFFFFFFFFFFFFF3CFF0A
:1009C000FFFFFFFFFFFFFFFFFFFFFFFFFFFFFFFF37
:1009D000FFFFFFFFFFFFFF3CF0001FFFFFFFFFFFD8
:1009E000FFFFFFFFFFFFFFFFFFFFFFFFFFFFFFFF17
:1009F00018E0001FFFFFFFFE0FFFFFFFFFFFFFFFDD
:100A0000FFFFFFFFFFFFFFFFFF81C0001FFFFFFF92
:100A1000FC07FFFFFFFFFFFFFFFFFFFFFFFFFFFFE1
:100A2000FFFFC3C0001FFFFFFFF843FFFFFFFFFFF3
:100A3000FFFFFFFFFFFFFFFFFFFFFFFFC1FFFFFF04
:100A4000FFFFF1F1C0FFFFFFFFFFFFFFFFFFFFFF11
:100A5000FFFFFFFFFFC3FFFFFFFFFFF3F9C0FFFF33
:100A6000FFFFFFFFFFFFFFFFFFFFFFFFFFFFC3FFD2
:100A7000FFFFFFFFF3F9FFFFFFFFFFFFFFFFFFFF98
:100A8000FFFFFFFFFFFFFFC3FFFFFFFFFFF3F9FFC4
:100A9000FFFFFFFFFFFFFFFFFFFFFFFFFFFFFFFF66
:100AA000C3FFFFFFFFFFF3F9FFFFFFFFFFFFFFFFA4
:100AB000FFFFFFFFFFFFFFFFFFC3FFFFFFFFFFF38E
:100AC000F9C3FFFFFFFFFFFFFFFFFFFFFFFFFFFF78
:100AD000FFFFC3FFFFFFFFFFF3F9C3FFFFFFFFFFB0
:100AE000FFFFFFFFFFFFFFFFFFFFFFC3FFFFFFFF52
:100AF000FFF3F9FFFFFFFFFFFFFFFFFFFFFFFFFF18
:100B0000FFFFFFFFC3FFFFFFFFFFF3F9FFFFFFFF43
:100B1000FFFFFFFFFFFFFFFFFFFFFFFFFFC3FFFF21
:100B2000FFFFFFF3F9FFFFFFFFFFFFFFFFFFFFFFE7
:100B3000FFFFFFFFFFFFC3FFFFFFFFFFF3F9C0FF52
:100B4000FFFFFFFFFFFFFFFFFFFFFFFFFFFFFFC3F1
:100B5000FFFFFFFFFFF3F9C0FFFFFFFFFFFFFFFFF6
:100B6000FFFFFFFFFFFFFFFFC3FFFFFFFFFFF3F9E3
:100B7000FFFFFFFFFFFFFFFFFFFFFFFFFFFFFFFF85
:100B8000FFC3FFFFFFFFFFF3F9FFFFFFFFFFFFFFC3
:100B9000FFFFFFFFFFFFFFFFFFFFC3FFFFFFFFFFA1
:100BA000F3F9FFFFFFFFFFFFFFFFFFFFFFFFFFFF67
:100BB000FFFFFFC1FFFFFFFFFFF3F9C3FFFFFFFFD1
:100BC000FFFFFFFFFFFFFFFFFFFFFFFFC0001FFF53
:100BD000FFFFF3F9C3FFFFFFFFFFFFFFFFFFFFFF73
:100BE000FFFFFFFFFFC0001FFFFFFFF3F9FFFFFF45
:100BF000FFFFFFFFFFFFFFFFFFFFFFFFFFFFE00023
:100C00001FFFFFFFF3F9FFFFFFFFFFFFFFFFFFFFE6
:100C1000FFFFFFFFFFFFFFF0001FFFFFFFF3F9FFE4
:100C2000FFFFFFFFFFFFFFFFFFFFFFFFFFFFFFFFD4
:100C3000FFFFFFFFFFFFF3F9C0FFFFFFFFFFFFFF15
:100C4000FFFFFFFFFFFFFFFFFFFFFFFFFFFFFFF3C0
:100C5000F9C0FFFFFFFFFFFFFFFFFFFFFFFFFFFFE9
:100C6000FFFFFFFFFFFFFFFFF3F9FFFFFFFFFFFFA6
:100C7000FFFFFFFFFFFFFFFFFFFFFFFFFFFFFFFF84
:100C8000FFF3F9FFFFFFFFFFFFFFFFFFFFFFFFFF86
:100C9000FFFFFFFFFFFFFFFFFFFFF319FFFFFFFF56
:100CA000FFFFFFFFFFFFFFFFFFFFFFFFFFFFFFFF54
:100CB000FFFFFFF319C3FFFFFFFFFFFFFFFFFFFF72
:100CC000FFFFFFFFFFFFFFFFFFFFFFFFF319C3FF62
:100CD000FFFFFFFFFFFFFFFFFFFFFFFFFFFFFFFF24
:100CE000FFFFFFFFFFF319FFFFFFFFFFFFFFFFFF06
:100CF000FFFFFFFFFFFFFFFFFFFFFFFFFFFFF319F6
:100D0000FFFFFFFFFFFFFFFFFFFFFFFFFFFFFFFFF3
:100D1000FFFFFFFFFFFFFFF319FFFFFFFFFFFFFFD5
:100D2000FFFFFFFFFFFFFFFFFFFFFFFFFFFFFFFFD3
:100D3000F319C0FFFFFFFFFFFFFFFFFFFFFFFFFFF4
:100D4000FFFFFFFFFFFFFFFFFFF319C0FFFFFFFFE4
:100D5000FFFFFFFFFFFFFFFFFFFFFFFFFFFFFFFFA3
:100D6000FFFFF319FFFFFFFFFFFFFFFFFFFFFFFF85
:100D7000FFFFFFFFFFFFFFFFFFFFFFF319FFFFFF75
:100D8000FFFFFFFFFFFFFFFFFFFFFFFFFFFFFFFF73
:100D9000FFFFFFFFF319FFFFFFFFFFFFFFFFFFFF55
:100DA000FFFFFFFFFFFFFFFFFFFFFFFFFFF319C381
:100DB000FFFFFFFFFFFFFFFFFFFFFFFFFFFFFFFF43
:100DC000FFFFFFFFFFFFF319C3FFFFFFFFFFFFFF61
:100DD000FFFFFFFFFFFFFFFFFFFFFFFFFFFFFFF32F
:100DE00019FFFFFFFFFFFFFFFFFFFFFFFFFFFFFFF9
:100DF000FFFFFFFFFFFFFFFFF319FFFFFFFFFFFFF5
:100E0000FFFFFFFFFFFFFFFFFFFFFFFFFFFFFFFFF2
:100E1000FFF319FFFFFFFFFFFFFFFFFFFFFFFFFFD4
:100E2000FFFFFFFFFFFFFFFFFFFFF319C0FFFFFF03
:100E3000FFFFFFFFFFFFFFFFFFFFFFFFFFFFFFFFC2
:100E4000FFFFFFF319C0FFFFFFFFFFFFFFFFFFFFE3
:100E5000FFFFFFFFFFFFFFFFFFFFFFFFF319FFFF94
:100E6000FFFFFFFFFFFFFFFFFFFFFFFFFFFFFFFF92
:100E7000FFFFFFFFFFE318FFFFFFFFFFFFFFFFFF85
:100E8000FFFFFFFFFFFFFFFFFFFFFFFFFFFFC31895
:100E90007FFFFFFFFFFFFFFFFFFFFFFFFFFFFFFFE2
:100EA000FFFFFFFFFFFFFF83183FFFFFFFFFFFFF75
:100EB000FFFFFFFFFFFFFFFFFFFFFFFFFFFFFFFF42
:100EC0000F1E1FFFFFFFFFFFFFFFFFFFFFFFFFFFE3
:100ED000FFFFFFFFFFFFFFFFFE3F1F8FFFFFFFFF33
:100EE000FFFFFFFFFFFFFFFFFFFFFFFFFFFFFFFF12
:100EF000FFFC7F1FC7FFFFFFFFFFFFFFFFFFFFFF9D
:100F0000FFFFFFFFFFFFFFFFFFFFF8FF1FE3FFFFF4
:100F1000FFFFFFFFFFFFFFFFFFFFFFFFFFFFFFFFE1
:100F2000FFFFFFF9FC07F3FFFFFFFFFFFFFFFFFFDE
:100F3000FFFFFFFFFFFFFFFFFFFFFFFFF1F001F1EA
:100F4000FFFFFFFFFFFFFFFFFFFFFFFFFFFFFFFFB1
:100F5000FFFFFFFFFFF3E010F9FFFFFFFFFFFFFFC1
:100F6000FFFFFFFFFFFFFFFFFFFFBFFFFFFFE3E00C
:100F700038F8FFFFFFFFFFFFFFFFFFFFFFFFFFFF4F
:100F8000FFFFFF1FFFFFFFE7C03C7CFFFFFFFFFFEE
:100F9000FFFFFFFFFFFFFFFFFFFFFFFE0FFFFFFF52
:100FA000E7801E3CFFFFFFFFFFFFFFFFFFFFFFFF8C
:100FB000FFFFFFFFFC07FFFFFFE7800E3CFFFFFF87
:100FC000FFFFFFFFFFFFFFFFFFFFFFFFFFF803FF34
:100FD000FFFFE7800E3CFFFFFFFFFFFFFFFFFFFF6C
:100FE000FFFFFFFFFFFFF001FFFFFFE780063CFF71
:100FF000FFFFFFFFFFFFFFFFFFFFFFFFFFFFFFE020
:1010000040FFFFFFE780003CFFFFFFFFFFFFFFFF08
:10101000FFFFFFFFFFFFFFFFC0E07FFFFFF7C00004
:101020007DFFFFFFFFFFFFFFFFFFFFFFFFFFFFFF52
:10103000FF81F03FFFFFF3E00079FFFFFFFFFFFFBD
:10104000FFFFFFFFFFFFFFFFFFFF03F81FFFFFF39F
:10105000E000F9FFFFFFFFFFFFFFFFFFFFFFFFFFC4
:10106000FFFFFE07FC0FFFFFF9F001F3FFFFFFFF9B
:10107000FFFFFFFFFFFFFFFFFFFFFFFC0FFE07FF6C
:10108000FFF9FC07F3FFFFFFFFFFFFFFFFFFFFFF7D
:10109000FFFFFFFFF81FFF03FFFFFCFE1FE7FFFF3F
:1010A000FFFFFFFFFFFFFFFFFFFFFFFFFFF03FFF1F
:1010B00081FFFFFE7FFFCFFFFFFFFFFFFFFFFFFF6F
:1010C000FFFFFFFFFFFFE07FFFC0FFFFFF3FFF9F2E
:1010D000FFFFFFFFFFFFFFFFFFFFFFFFFFFFFFC05F
:1010E000FFFFC07FFFFF8FFE3FFFFFFFFFFFFFFF00
:1010F000FFFFFFFFFFFFFFFFC0FFFFE07FFFFFC11C
:10110000F07FFFFFFFFFFFFFFFFFFFFFFFFFFFFF7E
:10111000FFC0F803E07FFFFFF000FFFFFFFFFFFFCE
:10112000FFFFFFFFFFFFFFFFFFFFE4F803E4FFFF08
:10113000FFFC07FFFFFFFFFFFFFFFFFFFFFFFFFFBA
:10114000FFFFFFFCF803E7FFFFFFFFFFFFFFFFFFCD
:10115000FFFFFFFFFFFFFFFFFFFFFFFFFCF803E7BD
:10116000FFFFFFFFFFFFFFFFFFFFFFFFFFFFFFFF8F
:10117000FFFFFFFFFFFCF803E7FFFFFFFFFFFFFF9D
:10118000FFFFFFFFFFFFFFFFFFFFFFFFFFFFFCF879
:1011900003E7FFFFFFFFFFFFFFFFFFFFCF3FFFFF63
:1011A000F3FFFFFFFFFFFFFCF803E7FFFFFFFFFF79
:1011B000FFFFFFFFFFCF3FFFF3F273FFFFFFFFFFD4
:1011C000FC000007FFFFFFFFFFFFFFFFFFFFCF3F18
:1011D000FFF3F273FFFFFFFFFFFC000007FFFFFFBD
:1011E000FFFFFFFFFFFFFFCF3FFFFFF3F3FFFFFF17
:1011F000FFFFFFFFFFFFFFFFFFFFFFFFFFFFFFFFFF
:10120000C0324033824099FFFFFFFFFFFFFFFFFF27
:10121000FFFFFFFFFFFFFFFFFFC0324C93327399C8
:10122000FFFFFFFFFFFFFFFFFFFFFFFFFFFFFFFFCE
:10123000FFFFCF324C92727399FFFFFFFFFFFFFF5A
:10124000FFFFFC0000000000007FFFCF324C9272D5
:1012500073C1FFFF8000000000000FFC00000000D1
:1012600000007FFFCF324C927273F9FFFF800000C5
:101270000000000FFC0000000000007FFFCF324C98
:10128000933273F9FFFF8000000000000FFC0000A4
:10129000000000007FFFCF38CC938270C3FFFF8037
:1012A00000000000000FFFFFFFFFFFFFFFFFFFFF39
:1012B000FFFFFFFFFFFFFFFFFFFFFFFFFFFFFFFF3E
:1012C000FFFFFFFFFFFFFFFFFFFFFFFFFFFFFFFF2E
:1012D000FFFFFFFFFFFFFFFFFFFFFFFFFFFFFFFF1E
:1012E000FFFFFFFFFFFFFFFFFFFFFFFFFFFFFFFF0E
:1012F000FFFFFFFFFFFFFFFFFFFFFFFFFFFFFFFFFE
:10130000FFFFFFFFFFFFFFFFFFFFFFFFFFFFFFFFED
:10131000FFFFFFFFFFFFFFFFFFFFFFFFFFFFFFFFDD
:10132000FFFFFFFFFFFFF3FFFFFFFFFFFFFFFFFFD9
:10133000FFFFFFFFFFFFFFFFFFFFFFFFFFFFFFE1DB
:10134000FFFFFFFFFFFFFFFFFFFFFFFFFFFFFFFFAD
:10135000FFFFFFFFFFFFFFFFE1FFFFFFFFFFFFFFBB
:10136000FFFFFFFFFFFFFFFFFFFFFFFFFFFFFFFF8D
:10137000FFC0FFFFFFFFFFFFFFFFFFFFFFFFFFFFBC
:10138000FFFFFFFFFFFFFFFFFFFFC47FFFFFFFFF28
:10139000FFFFFFFFFFFFFFFFFFFFFFFFFFFFFFFF5D
:1013A000FFFFFF8C7FFFFFFFFFFFFFFFFFFFFFFF40
:1013B000FFFFFFFFFFFFFFFFFFFFFFEF8E3FFFFF7E
:1013C000FFFFFFFFFFFFFFFFFFFFFFFFFFFFFFFF2D
:1013D000FFFFFFFFC71E3FFFFFFFFFFFFFFFFFFFF6
:1013E000FFFFFFFFFFFFFFFFFFFFFFFFFF871F1F45
:1013F000FFFFFFFFFFFFFFFFFFFFFFFFFFFFFFFFFD
:10140000FFFFFFFFFFFF923F1FFFFFFFFFFFFFFFF9
:10141000FFFFFFFFFFFFFFFFFFFFFFFFFFFFFF30AB
:101420003F8FFFFFFFFFFFFFFFFFFFFFFFFFFFFFFC
:10143000FFFFFFFFFFFFFFFE387FCFFFFFFFFFFF34
:10144000FFFFFFFFFFFFFFFFFFFFFFFFFFFFFFFFAC
:10145000FE787FE7FFFFFFFFFFFFFFFFFFFFFFFFBC
:10146000FFFFFFFFFFFFFFFFFFFEFCFFE7FFFFFFA8
:10147000FFFFFFFFFFFFFFFFFFFFFFFFFFFFFFFF7C
:10148000FFFFFCF8C0F3FFFFFFFFFFFFFFFFFFFFC1
:10149000FFFFFFFFFFFFFFFFFFFFFFFDF9C0F3FFAF
:1014A000FFFFFFFFFFFFFFFFFFFFFFFFFFFFFFFF4C
:1014B000FFFFFFFFF9F9FFF1FFFFFFFFFFFFFFFF56
:1014C000FFFFFFFFFFFFFFFFFFFFFFFFFFF3F1FF46
:1014D000F9FFFFFFFFFFFFFFFFFFFFFFFFFFFFFF22
:1014E000FFFFFFFFFFFFF3F3FFF8FFFFFFFFFFFF2B
:1014F000FFFFFFFFFFFFFFFFFFFFFFFFFFFFFFE714
:10150000E3C3FCFFFFFFFFFFFFFFFFFFFFFFFFFF46
:10151000FFFFFFFFFFFFFFFFE7E7C3FC7FFFFFFFCA
:10152000FFFFFFFFFFFFFFFFFFFFFFFFFFFFFFFFCB
:10153000FFE7C7FFFE7FFFFFFFFFFFFFFFFFFFFF8C
:10154000FFFFFFFFFC3F9FFFFFFFE3CFFFFE3FFFDB
:10155000FFFFFFFFFFFFFFFFFFFFFFFFFFF81F1F62
:10156000FFFFFFF38FFFFF3FFFFFFFFFFFFFFFFFC7
:10157000FFFFFFFFFFFFF18E1FFFFFFFF19FC0FF87
:101580009FFFFFFFFFFFFFFFFFFFFFFFFFFFFFF3D7
:10159000CE1FFFFFFFF81FC0FF9FFFFFFFFFFFFFF2
:1015A000FFFFFFFFFFFFFFFFF3CC3FFFFFFFFC3F0D
:1015B000FFFF9FFFFFFFFFFFFFFFFFFFFFFFFFFF9B
:1015C000FFF18C3FFFFFFFFE3FFFFFCFFFFFFFFF5D
:1015D000FFFFFFFFFFFFFFFFFFFFF81C7FFFFFFF85
:1015E000FE3FFFFFCFFFFFFFFFFFFFFFFFFFFFFFFC
:1015F000FFFFFFFC387FFFFFFFFE7FC3FECFFFFF33
:10160000FFFFFFFFFFFFFFFFFFFFFFFFFFF8FFFFF1
:10161000FFFFFE7FC3FCCFFFFFFFFFFFFFFFFFFFCA
:10162000FFFFFFFFFFFFF0FFFFFFFFFE7FFFFCCF8D
:10163000FFFFFFFFFFFFFFFFFFFFFFFFFFFFFFF1C8
:10164000FFFFFFFFFE7FFFF88FFFFFFFFFFFFFFFA2
:10165000FFFFFFFFFFFFFFFFE1FFFFFFFFFF3FFF78
:10166000F89FFFFFFFFFFFFFFFFFFFFFFFFFFFFFF1
:10167000FFE1FFFFFFFFFF1FC0F19FFFFFFFFFFF25
:10168000FFFFFFFFFFFFFFFFFFFFE3FFFFFFFFFF86
:101690001FC0E31DFFFFFFFFFFFFFFFFFFFFFFFF77
:1016A000FFFFFFC387FFFFFFFF8FFFC738FFFFFF6D
:1016B000FFFFFFFFFFFFFFFFFFFFFFFFC703FFFF6E
:1016C000FFFF8FFF8E7DFFFFFFFFFFFFFFFFFFFF8D
:1016D000FFFFFFFFFF8631FFFFFFFFC7FF9C77FF84
:1016E000FFFFFFFFFFFFFFFFFFFFFFFFFFFF8E7901
:1016F000FFFFFFFFE3FFF8E3FFFFFFFFFFFFFFFF39
:10170000FFFFFFFFFFFFFF0E79FFFFFFFFF1FFE18C
:10171000F7FFFFFFFFFFFFFFFFFFFFFFFFFFFFFFE1
:101720001E31FFFFFFFFF87F83BFFFFFFFFFFFFFBB
:10173000FFFFFFFFFFFFFFFFFE1F03FFFFFFFFFE97
:10174000000F1FFFFFFFFFFFFFFFFFFFFFFFFFFF78
:10175000FFFE3F87FFFFFFFFFF807FBFFFFFFFFF11
:10176000FFFFFFFFFFFFFFFFFFFFFFFFFFFFFFFF89
:10177000FFFFFFFFFFFFFFFFFFFFFFFFFFFFFFFF79
:10178000FFFFFFFFFFFFFFFFFFFFFFFFFFFFFFFF69
:10179000FFFFFFFFFFFFFFFFFFFFFFFFFFFFFFFF59
:1017A000FFFFFFFFFFFFFFFFFFFFFFFFFFFFFFFF49
:1017B000FFFFFFFFFFFFFFFFFFFFFFFFFFFFFFFF39
:1017C000FFFFFFFFFFFFFFFFFFFFFFFFFFFFFFFF29
:1017D000FFFFFFFFFFFFFFFFFFFFFFFFFFFFFFFF19
:1017E000FFFFFFFFFFFFFFFFFFFFFFFFFFFFFFFF09
:1017F000FFFFFFFFFFFFFFFFFFFFFFFFFFFFFFFFF9
:10180000FFFFFFFFFFF800000000000000000000E5
:10181000000000000000000000000000001FF800B1
:1018200000000000000000000000000000000000B8
:101830000000000000001FF8000000000000000091
:101840000000000000000000000000000000001F79
:10185000F800000000000000000000000000000090
:1018600000000000000000001FFFFFFFFFFFFFFF60
:10187000FFFFFFFFFFFFFFFFFFFFFFFFFFFFFFFF78
:10188000FFFFFFFFFFFFFFFFFFFFFFFFFFFFFFFF68
:10189000FFFFFFFFFFFFFFFFFFFFFFFFFFFFFFFF58
:1018A000FFFFFFFFFFFFFFFFFFFFFFFFFFFFFFFF48
:1018B000FFFFFFFFFFFFFFFFFFFFFFFFFFFFFFFF38
:1018C000FFFFFFFFFFFFFFFFFFFFFFFFFFFFFFFF28
:1018D000FFFFFFFFFFFFFFFFFFFFFFFFFFFFFFFF18
:1018E000FFFFFFFFFFFFFFFFFFFFFFFFFFFFFFFF08
:1018F000FFFFFFFFFFFFFFFFFFFFFFFFFFFFFFFFF8
:10190000FFFFFFFFFFFFFFFFFFFFFFFFFFFFFFFFE7
:10191000FFFFFFFFFFFFFFFFFFFFFFFFFFFFFFFFD7
:10192000FFFFFFFFFFFFFFFFFFFFFFFFFFFFFFFFC7
:10193000FFFFFFFFFFFFFFFFFFFFFFFFFFFFFFFFB7
:10194000FFFFFFFFFFFFFFFFFFFF2D000303050465
:10195000030406171000FD0BFD0BFE000000000144
:1019600073200500882523196A8B2B43429150145C
:101970003B8814455189EC10134525D29010002462
:1019800018C86B2AA3258B28428A15ADC408295292
:101990008948AC71400C0025216F8BB188C1C948C2
:1019A0002813456512E9880EA844EA80CA382293B4
:1019B0004A64D2D06418AC0026156B8BADAA93A1F3
:1019C0004C3899364956D42AC2115B6500270782E4
:1019D000FC270E01280AA36B665428FA2451290C0F
:1019E000A36D27249289BE5C24002A0AA6DC6A68BB
:1019F00022938C022B14298F30E39038240E091E79
:101A00008471481C128704012C09836A6524140917
:101A1000002D0744BA260E012E06428C25082F0EF3
:101A2000A56BE7D4626AC1985A4C2D08300F688BB9
:101A3000A9682289901F2522190900310A658BE9BE
:101A40002487914C3F3211688BA94A93894C2C9D75
:101A50000A69B4E1F4103313688B694A93894C2CFA
:101A6000A303E400226D6223013413698B29A78C40
:101A700012D9442652131D0E543940043510688B78
:101A8000292E62E5CB682CA61D4625003612688BF0
:101A9000A9681351902CA18C8A8C12918C04371058
:101AA000688B290E61E9543A954EA58B4300381294
:101AB000688B692CA36269441349848CA5110900C1
:101AC0003912688BA968228990589A9CC534916410
:101AD000460200000004FFFF0394186A896AE3A02D
:101AE00038641C1187C221614C18144545E143013B
:101AF00003A9206D892DCB52611C10930344728081
:101B0000480E10C90132A9281613CD42A143A800DE
:101B100003BC19695B2A6422994826928964229938
:101B2000687298D40172801C0003C013088B6A0E7F
:101B3000915030140C054331514C541B20302B76FE
:101B40008BB88871E0642407CA4471A84C22878E40
:101B5000E8089548A90EA858C611194D2A91D1A494
:101B6000A18965182C550020390BC49A6626922548
:101B7000D100203A0CC49A2664A2C944090020442A
:101B800011678BA9A3D2A8501A954685D23000219F
:101B9000220F89FA2A262A21892434498A242202FA
:101BA00017C77B68E68038200E08278946C4C548D9
:101BB0004C120BCA00220F20ED692E0E96034D2CFD
:101BC00013CBC432B14C2C13CBC432B14C2C13CB3D
:101BD000C432B1C45422111EEA6B2C0E1271480E8D
:101BE0009283E41039480E8A43E2A038240E8943D8
:101BF000E2800F2212082ACE300E03221A196989B8
:101C0000E92171401C12874466C15834140D85E5E2
:101C100000392406221E12ABAE7066935824260C9F
:101C2000CA22B1C86C02222B0DE75928D7A4E1FCC7
:101C3000B7210022480DAAAE7088423A9428A40029
:101C4000226012EAAEF001A1C3340E891E4671482B
:101C50001C022264122A8FF021D2E1540E9AC3E6AC
:101C6000B039EC302265122A8F30E2303A6C0E9394
:101C70000EA772C4C30025CA16878BA9A491582841
:101C800096128C441543B15062241A0300001200CE
:101C900005040506050507202400FB1EF91FFB00AF
:101CA00000000002802006008090092A2810AA5E09
:101CB0005B020968906188208608725032650C3298
:101CC0001E782009AA98840E11C41041CC20030567
:101CD000120A002B1238C310AD469DFFD6033FC039
:101CE000D4A8F3DF022C1348918B392A514619648A
:101CF00094410819841002002D09AA90D8097EA0E9
:101D0000002E08A5A090091E502F210D942E9A6830
:101D100088240A914421926888240A9144A59168F4
:101D200088240A914443249104003032D48BF06A11
:101D30009062C715430C29A68C82C828A888828A7D
:101D400028A884A2F47FAA84828A28A888828A2864
:101D5000A88C620A31A41877984206003116CCA3E9
:101D6000F07A8A310489071E504109448C29A7FE64
:101D7000FF0F3229D48BF16A5462E69507C278606E
:101D800008634C30A804834A28A9BCE2AC66DA692F
:101D900036766F1D7698710FFC030A3333D393F0B8
:101DA0005A126AE58D07C2784004634C30A78482DA
:101DB0008AAB9A59E82C94145A2AAD769C699653AA
:101DC000881D768A30C5880702798521550034310F
:101DD000D58BF0AA8E3B0DB16C69AA84A28828A984
:101DE0008882CA28A88C720A29A790624A29A694D8
:101DF000CA14624C21E514F2C07FACC07A040035ED
:101E000035D393EF1A1E10E201211E10E201211EAC
:101E100010A2B8FA84312524F240180F0871C809BD
:101E2000C698505071754E21769831E281301E0867
:101E3000A4215500363ED48BF06A925AA899471EC9
:101E400008C41423CC29C29C22CA2BCEB8F28A48DB
:101E5000A484351E180291138E31E11C86B8B45249
:101E6000090599509009E694618A190F84E20E538E
:101E7000A9003726D393F00AFE03A559AD348B99F8
:101E80006698691633CD30D30C3BCC34C34C33EC5D
:101E900030C30E33CDB093003841D48BF05A147256
:101EA000E581301E18E281218C31A2A0220A2AA2EB
:101EB000A0220A2AC218230E31E41D965272E5812F
:101EC000300E39A21C130C626829951862A8991368
:101ED0001E18E38150DC610400393ED48BF06A9017
:101EE00062C79507C278400C634C30C704834A3000
:101EF00068A5951862C884724E380489078660A167
:101F00000C254A31A438E3CAAB4439469453862998
:101F1000863CD3D052C9003A0C85AA90091E501FA6
:101F2000CC071400000004FFFF00001200060506A5
:101F300006050608373B00F732F332F700000000D1
:101F4000045820060000414A2A53DB86EFD5243886
:101F500002683806C6288CE4288EE4180EE5188E30
:101F6000C5188CC6088CA7088A284906233198E032
:101F7000083EE00714C221284772080911105111C8
:101F8000148F11188D3118CB311C09321CC9511C0A
:101F9000895118CC700C50700409002B1769EAC1E4
:101FA000628928C9FF7FD307FC03128928C9FFBFB4
:101FB00009002C214F34AFCA42291223311023319A
:101FC0009003319003398E03390EE4380EE4400C4F
:101FD000E440002D0A5132DB4BE01FD0012E0949AD
:101FE00072C14AE0074C2F3C973DB94EE80419D026
:101FF0000932A0B3E7804E90019D20033A7B0EE8A2
:102000000419D00932A0B3E7804E90019D20033A15
:102010007B0EE80419D00932A01364406790011DBB
:1020200010003062E22CBFD306B91C497AA8C65A08
:10203000B044431662391444311225291445211243
:1020400026211226191446111227111227111227C0
:10205000091427091487FEFF9C44489C44489C446B
:10206000489C445018654898844898845014A54862
:1020700094C45010E5588805D1126CB11AEA912425
:10208000E7421A003124556CC15326591465419A10
:10209000C329A0410A3EE00396601222E2311A648D
:1020A000511226FDFFFFFF033245A22CC15327B179
:1020B0009E68722C25433464333AA22918624996EB
:1020C0004159146159144169124169124169922CB4
:1020D00085295882A92EE55AACC5622AF68F6A284E
:1020E000A662514CC5AA96EB03FE0FC000335BE01D
:1020F0003CBFD3459920875AAC043BB46223BA81D4
:1021000031964149964059944061922069922069E4
:10211000922BCD522A656A98A9899E276A26478202
:1021200020C9992AE652AEE452AEB44B7264CEC4D2
:10213000504C22288A2228893230C6426C85766427
:1021400088C54C0E44250C00345BA51CC15389C9BD
:1021500018ACB95CD6AB82A8D88404C9840489843D
:102160000849940849840C09940C098410C9831403
:1021700089931489831849931849831C09931CC9AE
:102180009220C9822489922489822849922809921E
:102190002C09922CC99130C9F101FF0F88AA844BF8
:1021A000FF1D003549A13CBF53A123FA8F482EF5EE
:1021B000AF401445681025800CAEE8086FF086C665
:1021C0006084455104655982A45182A451B0F4C37E
:1021D0002467729240619440619241499681291826
:1021E000A22BB6234BAE857A204A69003674E22CC6
:1021F000BF5307B91C497AA8C65AB04443B48329CF
:10220000568852288A42284B32284C32245982A9B7
:10221000B0244B8E634988E65086C75084A850820C
:102220008948826AF88040780A4668922568922533
:102230006016256016ABA9D72881D22881D22881C3
:10224000D22881D22483B22883B228C39228C5829F
:102250002805532CC78664CAC5548E243917D2006A
:102260003745A13CBF53E0FF0110965C2A4BB914DF
:102270004BB9146BB1146BB1944BB1944BB1164B79
:10228000B1164BB156D5622D96622D9662ADAAC598
:102290005AAAC55A558BB5548BB5548BB5544CB509
:1022A000544CB54400386DE22CBF5346A124C75AA4
:1022B000B0443BB8C2233C82319881411861511629
:1022C000416114416114416114416114416114413F
:1022D0006194415114624196623196434BAE6692CD
:1022E0001C297A2A064336833196424996615194D5
:1022F0004161144161944071E8732AC6622E8509D8
:102300009684111AA3193CC22BB843532C479A1632
:1023100006003976E22CBFD306B91C49722AE65270
:1023200032643BB86231984249964151962161949A
:102330002161964069942071942071942071684EB7
:10234000D5548CC53081A234C1923401633CC2079C
:1023500004431524031528842428C633284743281A
:10236000CA7124590A536149960C09A30C099310A8
:102370008AA21449B2140AA21C4AC11C5A822D56C0
:10238000433D92E45C8803003A108998C14AE00713
:102390004C3F48FA800F980000000004FFFF000047
:1023A000652B11241FBECFEFD8E0DEBFCDBF27E0E5
:1023B000A8EFB1E001C01D92AD31B207E1F711E025
:1023C000A0E0B1E0E6E0FDE602C005900D92A83F76
:1023D000B107D9F711E1C1EDD1E104C02197FE01A8
:1023E0000E94CE33C03DD107C9F70E94342C0C9413
:1023F00081360C94000080915A0290915B02891BF7
:10240000990B089508950895AF92BF92CF92DF92ED
:10241000EF92FF920F931F93CF93DF936C017B0199
:102420008B01040F151FEB015E01AE18BF08C0172A
:10243000D10759F06991D601ED91FC910190F0819D
:10244000E02DC6010995892B79F7C501DF91CF9160
:102450001F910F91FF90EF90DF90CF90BF90AF90C2
:102460000895FC01538D448D252F30E0842F90E09A
:10247000821B930B541710F0CF960895019708957F
:10248000FC01918D828D981761F0A28DAE0FBF2F48
:10249000B11D5D968C91928D9F5F9F73928F90E09E
:1024A00008958FEF9FEF0895FC01918D828D98170D
:1024B00031F0828DE80FF11D858D90E008958FEF4A
:1024C0009FEF0895FC01918D228D892F90E0805C13
:1024D0009F4F821B91098F73992708958CEC92E08E
:1024E0000E94621221E0892B09F420E0822F0895D6
:1024F00080E090E0892B29F00E946E1281110C94EB
:1025000000000895FC01A48DA80FB92FB11DA35A96
:10251000BF4F2C91848D90E001968F739927848F03
:10252000A689B7892C93A089B1898C918370806426
:102530008C93938D848D981306C00288F389E02DC7
:1025400080818F7D80830895EF92FF920F931F9378
:10255000CF93DF93EC0181E0888F9B8D8C8D981356
:102560001AC0E889F989808185FF15C09FB7F89462
:10257000EE89FF896083E889F989808183708064AE
:1025800080839FBF81E090E0DF91CF911F910F91F9
:10259000FF90EF900895F62E0B8D10E00F5F1F4F08
:1025A0000F731127E02E8C8D8E110CC00FB607FC17
:1025B000FACFE889F989808185FFF5CFCE010E94A5
:1025C0008212F1CFEB8DEC0FFD2FF11DE35AFF4F7F
:1025D000F0829FB7F8940B8FEA89FB898081806233
:1025E000CFCFCF93DF93EC01888D8823B9F0AA89F0
:1025F000BB89E889F9898C9185FD03C0808186FDBE
:102600000DC00FB607FCF7CF8C9185FFF2CF80810C
:1026100085FFEDCFCE010E948212E9CFDF91CF91ED
:102620000895833081F028F4813099F08230A9F048
:1026300008958730A9F08830C9F08430B1F48091D2
:1026400080008F7D03C0809180008F778093800011
:10265000089584B58F7784BD089584B58F7DFBCFB1
:102660008091B0008F778093B00008958091B00082
:102670008F7DF9CF1F93CF93DF93282F30E0F9019F
:10268000E255FA4F8491F901E656FA4FD491F901D7
:10269000EA57FA4FC491CC23A9F0162F81110E945A
:1026A0001113EC2FF0E0EE0FFF1FE458FA4FA59145
:1026B000B4918FB7F894EC91111108C0D095DE2336
:1026C000DC938FBFDF91CF911F910895DE2BF8CF60
:1026D000CF93DF9390E0FC01E656FA4F24918A579E
:1026E0009A4FFC0184918823C9F090E0880F991FCC
:1026F000FC01EE58FA4FA591B491FC01E458FA4F51
:10270000C591D49161110DC09FB7F8948C9120951B
:1027100082238C938881282328839FBFDF91CF91C8
:102720000895623051F49FB7F8943C91822F8095C0
:1027300083238C93E8812E2BEFCF8FB7F894EC9105
:102740002E2B2C938FBFEACF3FB7F8948091520283
:1027500090915302A0915402B091550226B5A89BC6
:1027600005C02F3F19F00196A11DB11D3FBFBA2F23
:10277000A92F982F8827BC01CD01620F711D811DE3
:10278000911D42E0660F771F881F991F4A95D1F768
:1027900008958F929F92AF92BF92CF92DF92EF9265
:1027A000FF926B017C010E94A4134B015C01C114D8
:1027B000D104E104F104B9F00E94A4136819790965
:1027C0008A099B09683E73408105910580F321E0E9
:1027D000C21AD108E108F10888EE880E83E0981E3D
:1027E000A11CB11CE4CFFF90EF90DF90CF90BF9081
:1027F000AF909F908F900895EF92FF920F931F9349
:10280000FC01802F87018130A1F048F08230D1F0A7
:102810008330F9F01F910F91FF90EF900895808120
:102820009181DC01ED91FC91068CF78DE02D0995ED
:10283000F1CF80819181DC01ED91FC91048CF58DCB
:10284000E02DF5CF80819181621B730B6F5F7F4F0D
:10285000E8CF80819181421B530B4F5F5F4FEBCFDD
:10286000213069F038F0223079F0840F911D47FD56
:102870009A950895860F911D67FD9A950895841B7A
:10288000910947FD93950895861B910967FD9395DE
:102890000895213069F038F0223079F0861B9109D3
:1028A00067FD93950895840F911D47FD9A950895AE
:1028B000860F911D67FD9A950895841B910947FD28
:1028C000939508957F928F929F92AF92BF92CF92ED
:1028D000DF92EF92FF920F931F93CF93DF93EC0160
:1028E000162F842E9E84CF84D888D918712ED116A5
:1028F00008F47D2CE884F9840C89202F4C2D692D57
:102900008E819F810E9430145C01202F4C2D692DF7
:10291000C7010E944914AC01772051F0882071F062
:10292000EA84FB84272D30E0B501CE010E94FC1320
:102930001D1550F01D19C394912CD6CF8B89811190
:10294000F7CFEC84FD84EECF190D1E87CF86DF9183
:10295000CF911F910F91FF90EF90DF90CF90BF909C
:10296000AF909F908F907F900895DC011E964C91C0
:102970001E97ED91FC911197249130E0042E02C036
:10298000359527950A94E2F7842F860F883068F0F2
:1029900031961196FC93EE93E49198E0941B01C05C
:1029A000EE0F9A95EAF72E2B88501E968C938FEF98
:1029B0009FEF01C0880F6A95EAF7809582230895FA
:1029C000CF93C62F0E94B514C15021E030E001C062
:1029D000220FCA95EAF7821BCF910895FC01E60FFA
:1029E000F11D849190E0982F88273196E4918E0F05
:1029F000911D0895CF93DF9320917B0330917C0349
:102A00002817390709F472C0EC0190937C03809376
:102A10007B0310928C03FC01849180938E0331968A
:102A2000E491E0938F03FE013296E491E0939003EA
:102A3000FE013396E491E0939103FE013496E49114
:102A4000E0939203FE013596E491E0939303FE0137
:102A50003696E491E0939403FE013796E491E09377
:102A60009503FE013896E491E0939603FE013996B2
:102A7000E491E0939703FE013A96E491E093980382
:102A8000FE013B96E491E0939903FE013C96E491AC
:102A9000E0939A03FE013D96E491E0939B03FE01CF
:102AA0003E96E491E0939C03FE013F96E491E0930F
:102AB0009D03FE017096E491E0939E0361E1CE01D7
:102AC0000E94EE149093A00380939F0363E1CE01D4
:102AD0000E94EE149093A2038093A10365E1CE01BE
:102AE0000E94EE149093A4038093A303DF91CF91EF
:102AF00008950895FC016370668B84819581268119
:102B00003781613039F0633029F0918780873387CE
:102B100022870895318720879387828708952F928F
:102B20003F924F925F926F927F928F929F92AF925D
:102B3000BF92CF92DF92EF92FF920F931F93CF93AA
:102B4000DF93CDB7DEB76A970FB6F894DEBF0FBE3E
:102B5000CDBF9A8F898F7A8369834A01D22E1887D5
:102B60000F833701BC2CDC0159962D913C915A976B
:102B70002115310509F015C118968D919C91199771
:102B8000681779070CF0D7C11A968D919C91481758
:102B900059070CF0D0C14C2C512CB6E0CB9E600DE7
:102BA000711D11247C876B87161617060CF0C3C1A4
:102BB000EA2DF0E0FA87E98793E0EE0FFF1F9A9580
:102BC000E1F7F88BEF87CF01840F951F18161906D0
:102BD0000CF0B1C1A98DBA8D58968C91811104C0A9
:102BE000BFEABD1508F4D394A98DBA8DED91FC917F
:102BF00011970284F385E02DCD010995B5E0DB9EA8
:102C0000C0011124E981FA81FC83EB83312C212C52
:102C10009C012E583F4F388F2F8B4A2D50E05E8BF2
:102C20004D8BEF89F88DE20DF31D44919E828D82CC
:102C3000D12CC12C69817A81620D731D7A8B698BCD
:102C4000842F90E09C8B8B8BE98DFA8DA081B181D4
:102C500040FF82C0F1E0BF126FC0AF126DC01C9682
:102C6000ED91FC912F813885A4014C0D5D1D698982
:102C70007A89898D9A8D0995EB89FC89F595E79577
:102C80004E2F5FEFC51AD50A6D817E818D899E8991
:102C9000680F791F7E836D8398E0C916D10481F691
:102CA000AFEF2A1A3A0AEB81FC81E40DF51DFC8393
:102CB000EB83F5E02F16310409F0B3CF2F8138856F
:102CC00026153705B9F0A98DBA8DED91FC91B1E0CB
:102CD000BB1257C0AB1255C069817A816B5F7F4FC1
:102CE0000088F189E02D830128E030E0A401898D7E
:102CF0009A8D0995A98DBA8DED91FC911197068851
:102D0000F789E02DCD016A960FB6F894DEBF0FBEAD
:102D1000CDBFDF91CF911F910F91FF90EF90DF908A
:102D2000CF90BF90AF909F908F907F906F905F906B
:102D30004F903F902F9009941E96ED91FC91EF805B
:102D4000F88409851A8592014D815E816B817C81B1
:102D5000898D9A8D099590CF2F8138852615370555
:102D600009F48ACF31E0B31207C0A31205C01C9644
:102D7000ED91FC91930178CF1E96ED91FC9173013A
:102D8000E0CF6B857C85641975090684F785E02D95
:102D900073010F8518899201A401898D9A8D099577
:102DA000A9CFF90134969491329745915491D91A4B
:102DB000B7E0DB9E400D511D1124F901259134919E
:102DC0003C8B2B8BFA0125903490FA01329674904B
:102DD00031963491398B329664903196449041E02B
:102DE0004C1518F04A1508F07FC0662D062C000C13
:102DF000770B7C836B83842D042C000C990B9E83B2
:102E00008D83A98DBA8DED91FC9111970284F38584
:102E1000E02DCD010995512CD12CC12CEA2DF0E0EB
:102E2000FA87E9872B2D30E03C872B87A401440DDE
:102E3000511D47FC5A95588F4F8B69817A81660DD9
:102E4000711D67FC7A957E876D877989C71608F0B2
:102E500051CF2C2D30E04D815E81420F531FA9854B
:102E6000BA854A9FC0014B9F900D5A9F900D112427
:102E7000FC01E80DF91DF88BEF87852D612C4F893A
:102E8000588D420F531F5E8B4D8B671408F050C056
:102E900044244394480E877041F4C1010196EB89A4
:102EA000FC89E20DF31DD4901C01D7FE19C0A98D39
:102EB000BA8DED91FC91662D70E0B1E0BB1219C0A6
:102EC000AB1217C02D853E85620F731F0484F585F4
:102ED000E02D2F8138854D895E89898D9A8D0995E0
:102EE000DD0C6394842DD1CF1E821D821C821B8237
:102EF00088CF4B815C81640F751FAB85BC856A9F51
:102F0000C0016B9F900D7A9F900D112469817A8189
:102F1000680F791F0684F785E02DEF80F884098516
:102F20001A859D014F855889898D9A8D0995D8CF2D
:102F3000570CC3948ACF6A960FB6F894DEBF0FBEC3
:102F4000CDBFDF91CF911F910F91FF90EF90DF9058
:102F5000CF90BF90AF909F908F907F906F905F9039
:102F60004F903F902F9008958F929F92AF92CF9263
:102F7000EF92FF920F931F93CF93DF93EC01262FD5
:102F8000898D9A8D009709F051C06A30D1F41D8661
:102F90001C868D8948E0849F900111248E859F8531
:102FA000820F931F9F878E8781E090E0DF91CF9102
:102FB0001F910F91FF90EF90CF90AF909F908F90C7
:102FC00008956D3089F3CC88AD888F898823C1F04E
:102FD0008C859D8536E0C39E800D911D112448850A
:102FE00059854817590764F44E855F851D861C86F0
:102FF00038E0A39EC0011124840F951F9F878E8700
:10300000EA88FB88088919894E855F856C857D85EE
:10301000CE010E948F152C898C859D8546E0249FCA
:10302000800D911D11249D878C87BECF6A3069F475
:103030001D861C86FC013896E4912D898E859F851E
:10304000E29F800D911D1124ADCF6D3009F4ACCFFE
:10305000FC0134963491631708F4A6CF3296E491BC
:10306000E61708F4A1CFFC01329685909490462F84
:10307000431B342F47E0349F800C911C1124F40132
:10308000329634913196E4913323A9F1EE2399F1EC
:10309000CC88F4013596E491AD884F89442301F141
:1030A0000E2E000CFF0BE30FF11DCE9EA001CF9E54
:1030B000500D11246C857D85460F571F68857985D5
:1030C000641775076CF44E855F851D861C86FC01B0
:1030D0003896E491AE9E400D511D11245F874E87B6
:1030E000EA88FB88088919894E855F856C857D850E
:1030F000CE010E948F15F4013496E4912C898C85C1
:103100009D85E29F800D911D11248DCF6F927F923E
:103110008F929F92AF92BF92CF92DF92EF92FF92E7
:103120000F931F93CF93DF93EC016B015A01390189
:103130004801E881F9810284F385E02D0995E88151
:10314000F9810288F389E02D87019301A501B60179
:10315000CE010995A501480D591D41505109E8813D
:10316000F9810288F389E02D9301B601CE0109951A
:10317000E881F9810088F189E02D9401A501B6016B
:10318000CE010995C60CD71CB60161507109E881C2
:10319000F9810088F189E02D9401A501CE010995FE
:1031A000E881F9810688F789E02DCE01DF91CF9182
:1031B0001F910F91FF90EF90DF90CF90BF90AF9055
:1031C0009F908F907F906F9009946F927F928F92D3
:1031D0009F92AF92BF92CF92DF92EF92FF920F93A6
:1031E0001F93CF93DF935C01EB016A014901380122
:1031F0008701DC01ED91FC916217730719F56416E4
:1032000075062CF0962D872D3A01C92ED82E9601E1
:10321000261937092F5F3F4F048CF58DE02DA30150
:10322000BE01C5010995DF91CF911F910F91FF90CC
:10323000EF90DF90CF90BF90AF909F908F907F9056
:103240006F9008954615570591F42617370724F017
:10325000892D4B01C22FD82F9E01281939092F5FC4
:103260003F4F068CF78DE02DA601B401DACF028422
:10327000F385E02D0995D501ED91FC910488F58940
:10328000E02D83019401A601BE01C5010995D50178
:10329000ED91FC910688F789E02DC501DF91CF9172
:1032A0001F910F91FF90EF90DF90CF90BF90AF9064
:1032B0009F908F907F906F900994EF92FF920F9361
:1032C0001F93DC011A960D911C911B9718962D9156
:1032D0003C911997ED91FC9100A0F1A1E02D7B01AB
:1032E00050E040E070E060E009951F910F91FF9081
:1032F000EF9008954F925F926F927F928F929F927C
:10330000AF92BF92CF92DF92EF92FF920F931F93F3
:10331000CF93DF936C012B015A0139014801DC0185
:10332000ED91FC910284F385E02D0995E201640C96
:10333000751CD601ED91FC91C615D7055CF400888B
:10334000F189E02D87019401A501BE01C60109950F
:103350002196EFCF0688F789E02DC601DF91CF9146
:103360001F910F91FF90EF90DF90CF90BF90AF90A3
:103370009F908F907F906F905F904F9009948F9265
:103380009F92AF92BF92CF92DF92EF92FF920F93F4
:103390001F93CF93DF93EC015B014A016901E88140
:1033A000F9810284F385E02D099595012C0D3D1DD1
:1033B00021503109E881F9810488F589E02D7801EF
:1033C0008401A401B501CE010995E881F98106883F
:1033D000F789E02DCE01DF91CF911F910F91FF90E2
:1033E000EF90DF90CF90BF90AF909F908F90099417
:1033F0008F929F92AF92BF92CF92DF92EF92FF9205
:103400000F931F93CF93DF93EC015B014A01690196
:103410007801E881F9810284F385E02D0995C80CD3
:10342000D91C860101501109E881F9810488F589C8
:10343000E02D9501A401B501CE010995E881F9813E
:103440000688F789E02DCE01DF91CF911F910F9172
:10345000FF90EF90DF90CF90BF90AF909F908F90B4
:1034600009940895EF92FF920F931F93DC01ED9161
:10347000FC9100A0F1A1E02D09951F910F91FF9003
:10348000EF9008950F931F93DC01ED91FC91068C52
:10349000F78DE02D09951F910F9108950F931F93BC
:1034A000DC01ED91FC91048CF58DE02D09951F91C7
:1034B0000F910895DC01ED91FC910084F185E02DE0
:1034C00009942F923F924F925F926F927F928F92C8
:1034D0009F92AF92BF92CF92DF92EF92FF920F93A3
:1034E0001F93CF93DF9300D000D000D0CDB7DEB7CD
:1034F0003C016A013E832D83FC82EB825801A41AB1
:10350000B50AB7FE03C0B194A194B1088D809E8026
:10351000861A970A97FE03C09194819491088A14A1
:103520009B045CF0902F812F0D811E819D838E83E3
:103530009C2D8D2D6B01692F782F0C151D055CF0CE
:103540009D818E817E836D83692F782F902F812FAF
:103550008601C92ED82E1601201A310A2B012D8181
:103560003E81421A530A57FE03C0519441945108B8
:10357000710137FE03C03FEFE31AF30AF594E794B5
:103580008D819E81861797075CF5A1E0B0E0BA8334
:10359000A983C016D1064CF1D301ED91FC910484AE
:1035A000F585E02D2B813C81A8016D817E818A14F7
:1035B0009B041CF04D815E81B801C3010995E4189C
:1035C000F508F7FE0AC02D813E8189819A81280F76
:1035D000391F3E832D83E20CF31C0F5F1F4FD9CFA1
:1035E0002FEF3FEF3A832983D4CF26960FB6F89476
:1035F000DEBF0FBECDBFDF91CF911F910F91FF9026
:10360000EF90DF90CF90BF90AF909F908F907F9082
:103610006F905F904F903F902F9008951F93CF939E
:10362000DF93EC01162FE881F9810680F781E02D08
:103630000995E881F9810288F389E02D61E0CE01E6
:103640000995E881F9810484F585E02D612FCE018B
:10365000DF91CF911F910994CF93DF93EC018D857A
:1036600087FD1BC09D899923D9F060E00E943A1321
:1036700061E08D850E9468136D8D7E8D90E080E005
:103680000E94C91362E08D850E94681368EC70E0A7
:1036900080E090E00E94C9131C8EDF91CF910895C5
:1036A00061E00E943A1361E08D850E94681364E135
:1036B00070E080E090E00E94C91360E08D850E9478
:1036C0003A136D8D7E8D90E080E00E94C91361E019
:1036D0008D850E943A13DACFEF920F931F93DC018E
:1036E000ED91FC910280F381E02DE12C04E110E0EA
:1036F00021E009951F910F91EF90089508958CBDD9
:103700009DBD089520912A02260F3327331F2132B1
:103710003105ECF42091A202FC0190E080E024301D
:1037200069F082E00895A0912A022191AC01465FE0
:103730005D4FA40FB52FB11D2C930196861798F3FA
:1037400080912A02680F60932A0280E0089581E048
:1037500008951092A20281E08093A10210927C024F
:1037600061E082E10E943A1361E083E10E943A1332
:10377000E9EBF0E080818E7F808380818D7F808384
:1037800088E48093B80085E48093BC000895CF93CB
:10379000DF9391E0909309028823B9F0C091B800BB
:1037A000D091BA008091BC008A7B8093BC0060E01D
:1037B00082E10E943A1360E083E10E943A130E9482
:1037C000A91BD093BA00C093B800DF91CF910895A0
:1037D000E0915B0280915A02E81730F4F0E0E45A7D
:1037E000FD4F808190E008958FEF9FEF08959091B5
:1037F0005B0280915A022FEF3FEF981748F4E92FB0
:10380000F0E0E45AFD4F208130E09F5F90935B022F
:10381000C9010895CF92DF92EF92FF920F931F9309
:10382000CF93DF937C01CB018A012091CB0222232D
:1038300089F0EB016B01C40ED51ECC15DD0569F0D6
:103840006991D701ED91FC910190F081E02DC701C4
:103850000995F3CF642F0E94821BC801DF91CF919D
:103860001F910F91FF90EF90DF90CF900895CF932D
:10387000DF931F92CDB7DEB769832091CB0222235D
:10388000F9F02091C802203258F021E030E0FC012C
:103890003383228390E080E00F90DF91CF910895F1
:1038A0008091C902E82FF0E0E855FD4F998190839F
:1038B0008F5F8093C9028093C80281E090E0ECCFD3
:1038C00061E0CE0101960E94821BF7CFCF92DF927A
:1038D000EF92FF920F931F93CF9391E09093CB02BF
:1038E00090E49093CA021092C9021092C802682F05
:1038F00089E693E00E94371CC091C802C13208F0EB
:1039000091C00E94A4136B017C018091A2028111DD
:1039100064C082E08093A20281E08093A1028FEFD5
:103920008093A00210929F02C0939E02A8EAB2E088
:10393000EEE7F2E080E0C81383C010927D02809130
:103940007D02806880937D0280917C02813009F045
:103950007BC010927C020E94A4136B017C018091B9
:103960007D028093BB008091A4029091A502A0915A
:10397000A602B091A702892B8A2B8B2B99F00E946B
:10398000A4130091A4021091A5022091A6023091E7
:10399000A7026C197D098E099F09061717072807CA
:1039A0003907E0F18091BC0083FDD9CF85EC80938D
:1039B000BC000E94A4136B017C018091A2028230A2
:1039C00009F444C08091A0028F3F61F18091A00270
:1039D000803241F18091A00225C08091A402909193
:1039E000A502A091A602B091A702892B8A2B8B2B4E
:1039F00009F48BCF0E94A4130091A4021091A50298
:103A00002091A6023091A7026C197D098E099F09A9
:103A1000061717072807390708F077CF8091A30208
:103A20000E94C71B1092C9021092C8021092CB02CA
:103A3000CF911F910F91FF90EF90DF90CF9008955D
:103A40009D9191938F5F77CF85EEB1CF8091A40246
:103A50009091A502A091A602B091A702892B8A2B72
:103A60008B2B09F4AACF0E94A4130091A4021091F9
:103A7000A5022091A6023091A7026C197D098E093A
:103A80009F09061717072807390708F096CFC6CFF2
:103A9000CF93CFB7F89480910802811127C0E0E955
:103AA000F5E08491E4EAF5E09491E82FF0E0EE0F80
:103AB000FF1FEE58FA4FA591B491EC91E92321F440
:103AC00061E08AE00E943A1361E08AE00E94681394
:103AD0008CB580618CBD8CB580648CBD61E08DE05F
:103AE0000E94681361E08BE00E94681380910802D5
:103AF0008F5F80930802CFBFCF9108958F929F92DE
:103B0000AF92BF92EF920F931F93CF93DF93EC018D
:103B10004A015B01288F298FED8A1A8E1B8E1C8E1D
:103B20001E8F0D8F81149104A104B10409F465C0A6
:103B3000E091DC02F091DD0282E08083811481EE6D
:103B40009806A104B104A1F060E079E08DE390E073
:103B5000A50194010E94983321503109410951096E
:103B60005695479537952795211580E13807A8F098
:103B7000E091DC02F091DD02108260E874E88EE1F1
:103B800090E0A50194010E94983321503109410928
:103B900051095695479537952795E091D802F091B0
:103BA000D9023083E091DA02F091DB022083109297
:103BB000E402E091E002F091E10286E08083E0918E
:103BC000DE02F091DF02808180618083E091DE027D
:103BD000F091DF02808188608083E091DE02F091C5
:103BE000DF02808180688083E091DE02F091DF0255
:103BF00080818F7D808381E08C8B8B8587FD07C0E2
:103C000061E00E943A1361E08B850E9468138C8505
:103C100087FD07C061E00E943A1361E08C850E9435
:103C20006813CE010E942C1B8E8587FD03C060E0C7
:103C30000E946813DF91CF911F910F91EF90BF9079
:103C4000AF909F908F900C94481D0F931F93CF932C
:103C5000DF93FC0177FD92C0808591856817790715
:103C60000CF08CC057FD8AC0A285B3854A175B074C
:103C70000CF084C0DF01A45ABC4FAC91AA2331F0F0
:103C80008C01061B170BB8016150710986898230BF
:103C900009F479C0833009F487C0813041F484810C
:103CA0009581841B950BAB01BC0161507109DF014B
:103CB000A859BC4F8D919C911197681B790B77FD8A
:103CC0005DC014960D90BC91A02D6A177B0708F07B
:103CD00055C0EF01C659DC4F88819981481B590BAB
:103CE00057FD4CC02496888199814817590708F0E0
:103CF00045C0289788819981249708811981809FE0
:103D0000E001819FD00D909FD00D11244C1B5D0BC5
:103D1000EF01C35ADC4FC881CC2331F0EC0121976D
:103D20008E01041B150BA80157FD28C04817590721
:103D300028F583E0B695A7958A95E1F7A49FC00181
:103D4000A59F900DB49F900D1124AB01A3E0559554
:103D50004795AA95E1F7840F951FE80FF91F42AD2B
:103D6000609570956770772781E090E001C0880FBB
:103D70006A95EAF7232B09F1842B82AFDF91CF916B
:103D80001F910F91089584819581DC01A61BB70BCB
:103D9000BD0161507109868197818C01041B150B4F
:103DA000A8014150510983CF86819781861B970BCB
:103DB000BA01AC01415051097ACF80958423DDCFFF
:103DC00021E0672B09F420E02195FC01FA96865A40
:103DD0009C4F2193E817F907E1F70895CF92DF92FE
:103DE000EF92FF920F931F93CF93DF936C01EB0140
:103DF0007B01E40EF51E10E000E0CE15DF0561F05A
:103E00006991D601ED91FC910190F081E02DC60100
:103E10000995080F191FF1CFC801DF91CF911F91AC
:103E20000F91FF90EF90DF90CF9008959F92AF9207
:103E3000BF92CF92DF92EF92FF920F931F93CF9397
:103E4000DF93EC01662359F08FA9811130C06C3FDC
:103E5000A0F085E08FAB617070E07EAB6DAB81E070
:103E600090E0DF91CF911F910F91FF90EF90DF9045
:103E7000CF90BF90AF909F900895683F20F084E06E
:103E80008FAB6370E9CF603F20F083E08FAB67704A
:103E9000E3CF603E20F082E08FAB6F70DDCFE62E87
:103EA000F12C603C98F081E08FAB6F71D5CF8150E1
:103EB0008FABEDA8FEA836E0EE0CFF1C3A95E1F7BB
:103EC0006F73E62AFEAAEDAA8111C9CF2AE0E21695
:103ED000F10491F41AAA19AA88A5082E000C990BCE
:103EE00029A5821B910927FD93952BA93CA9820F37
:103EF000931F9CAB8BABB3CF8DE0E816F10419F4A4
:103F00001AAA19AAACCFEEEFEE16EFEFFE0608F0F4
:103F1000A6CF8BA99CA929A93AA93B872A879D8767
:103F20008C878E819F814796FFEFEF16F10411F089
:103F300008F097C021E6E216F104F8F02CA53DA5A3
:103F4000820F931F9C012F5F3F4FF9014491411154
:103F50001BC090E080E0288D213039F208F4ADC01C
:103F6000223009F4B1C0233009F079CF2BA93CA944
:103F7000281B390B3CAB2BAB72CFE1E4EE16F104FE
:103F800008F32AA53BA5DCCFFC0144914E151F0484
:103F900009F062C002960097E1F26E01F4E0CF0EE4
:103FA000D11C86010C5F1F4F998788871E8A6D8DF3
:103FB000C8010E94B5148C8B6E8DC8010E94B51487
:103FC000B82E8D8B6F8DC8010E94E014A82E68A1B9
:103FD000C8010E94E014E82E69A1C8010E94E01403
:103FE000F82E8C891816A4F5988CEB0CE194292DE9
:103FF0004E2D6A2D8A859B850E9430149B878A8767
:10400000292D4E2D6A2D8C859D850E9449149D87F2
:104010008C871A8A1B8A6B8DC8010E94B514A82E42
:104020006C8DC8010E94B514E82E40E06A2DC601CF
:104030000E94621441E06E2DC6010E94621461E08C
:10404000C8010E94B5148111F0CF8B898B151CF328
:104050008F2DFF0C990B7FCFF9012491820F911DB9
:1040600071CF0EA51FA5080F191F680160E0C601DA
:104070000E94EE14080F191F62E0C6010E94EE14A0
:10408000F4E0CF0ED11C8E159F0580F3F8018491CA
:1040900090E0982F88273196E4918E2B009709F4B1
:1040A00058CFE816F90619F4C801039674CFF80141
:1040B0003296E4910E0F111DE9CF29A93AA9820F7A
:1040C000931F9AAB89ABCBCE29A93AA9281B390BF0
:1040D0003AAB29ABC4CE08956F927F928F929F9294
:1040E000AF92BF92CF92DF92EF92FF920F931F9306
:1040F000CF93DF93CDB7DEB7A989BA89FC01608081
:104100007180FD89FF93FC89FF93FB89FF93BF9327
:10411000AF93D3011A96ED91FC9109950F900F90F2
:104120000F900F900F90DF91CF911F910F91FF9003
:10413000EF90DF90CF90BF90AF909F908F907F9047
:104140006F9008958F92AF92CF92EF92FF920F935C
:104150001F93CF93DF93CDB7DEB7DC01ED91FC91D8
:104160000084F185E02D0995DF91CF911F910F918A
:10417000FF90EF90CF90AF908F900895DC01ED917C
:10418000FC910680F781E02D09948EBD00000DB4EE
:1041900007FEFDCF8EB508951F93CF93DF93EC01FB
:1041A000162F8E899F890E947F1B8B8587FD03C0F8
:1041B00060E00E943A13812F0E94C5208B8587FD05
:1041C00006C061E0DF91CF911F910C943A13DF910B
:1041D000CF911F9108951F93CF93DF93EC01162F7A
:1041E0008E899F890E947F1B8C8587FD03C060E0BC
:1041F0000E943A138B8587FD03C060E00E943A134A
:10420000812F0E94C5208B8587FD03C061E00E943D
:104210003A138C8587FD06C061E0DF91CF911F9135
:104220000C943A13DF91CF911F9108958F929F9232
:10423000AF92BF92CF92DF92EF92FF920F931F93B4
:10424000CF93DF93EC015B017A01490161E10E94A8
:10425000EB2063E0CE010E94CC2064E4CE010E94FA
:10426000EB20650183E0D694C7948A95E1F76C2D25
:10427000CE010E94CC20B401615071096A0D7B1DF2
:1042800093E0769567959A95E1F7CE010E94CC2050
:1042900065E4CE010E94EB206E2DCE010E94CC2061
:1042A0006F2DCE010E94CC206FEF600F6E0DCE01FE
:1042B0000E94CC20015011090E0D1F1D612FCE014F
:1042C0000E94CC206EE4CE010E94EB206C2DCE012A
:1042D0000E94CC206FE4CE010E94EB206E2DCE0117
:1042E0000E94CC206F2DCE01DF91CF911F910F91B5
:1042F000FF90EF90DF90CF90BF90AF909F908F9006
:104300000C94CC200F931F93CF93DF93EC018C8DF3
:10431000882319F0CE010E942C1B6AE070E080E037
:1043200090E00E94C91362E1CE010E94EB206AE096
:1043300070E080E090E00E94C91361E0CE010E942D
:10434000EB2067ECCE010E94CC2060E0CE010E9401
:10435000CC2060E0CE010E94CC206CE3CE010E9414
:10436000EB2065E0CE010E94CC2068E1CE010E94E6
:10437000EB2060E8CE010E94CC2067E3CE010E94D2
:10438000EB2060E0CE010E94CC2060E0CE010E94D4
:10439000CC2060E0CE010E94CC2060E0CE010E94E3
:1043A000CC206FEFCE010E94CC2060E0CE010E94B5
:1043B000CC2060E0CE010E94CC2060E0CE010E94C3
:1043C000CC2060E0CE010E94CC2061E0CE010E94B2
:1043D000CC2008EC10E028EC30E050E040E070E049
:1043E00060E0CE010E941621DF91CF911F910F91C5
:1043F0000895FF920F931F93CF93DF938C01F42EB8
:104400000E94EB20D0E0C0E06F2DC8010E94CC20BC
:104410002196C83883E1D807B9F7DF91CF911F9172
:104420000F91FF900895CF93DF93C82FD62F60E0B0
:1044300086E00E943A1380E28C0FC03238F08FE1A0
:104440008C0F833088F0CF3F79F08C2F0E94C520ED
:10445000C82F8D2F0E94C52061E086E00E943A138C
:104460008C2FDF91CF9108958C2F0E94C520C82FEB
:10447000F3CFCF93C82F60E086E00E943A138C2FD1
:104480000E94C52080E00E94C520C82F61E086E020
:104490000E943A138C2FCF910895EF92FF920F93C1
:1044A0001F93CF93DF93C82FF62EE72ED42F86309D
:1044B00019F080F4823080F483E00E943922D2E047
:1044C000D80F60E086E00E943A138AE28C0F0E94C7
:1044D000C52002C0873071F00F2D1E2DD15080F401
:1044E00061E086E0DF91CF911F910F91FF90EF90F7
:1044F0000C943A1360E086E00E943A1380EAE7CF1A
:10450000F80181918F010E94C520E8CF90E080E002
:1045100008958F929F92AF92BF92CF92DF92EF92C7
:10452000FF921F93CF93DF930E94A4136B017C0132
:104530008091A202811165C081E08093A2028093E4
:10454000A1029FEF9093A00210929F0292E090939D
:104550009E0280937D0280917D02806880937D021F
:1045600080917C02813009F089C010927C020E9407
:10457000A4136B017C0180917D028093BB0080912C
:10458000A4029091A502A091A602B091A702892B46
:104590008A2B8B2BA1F00E94A4138090A4029090F0
:1045A000A502A090A602B090A7026C197D098E0901
:1045B0009F0986169706A806B90608F443C080919D
:1045C000BC0083FDD8CF85EC8093BC000E94A4136F
:1045D0006B017C018091A202813009F451C080916D
:1045E0009F02D3E0833010F4D0919F02AEE7B2E097
:1045F000ECE5F2E080E08D1751F19D9191938F5F92
:10460000FACF8091A4029091A502A091A602B09148
:10461000A702892B8A2B8B2B09F48ACF0E94A41323
:104620008090A4029090A502A090A602B090A7024C
:104630006C197D098E099F0986169706A806B9068A
:1046400008F076CF8091A3020E94C71BD0E01092A1
:104650005B02D0935A0280915B02D81799F189E6E8
:1046600093E00E94F71BC82F89E693E00E94F71B96
:10467000182F89E693E00E94F71BEDCF85EEA4CFBB
:104680008091A4029091A502A091A602B091A702E8
:10469000892B8A2B8B2B09F49DCF0E94A413809029
:1046A000A4029090A502A090A602B090A7026C1957
:1046B0007D098E099F0986169706A806B90608F097
:1046C00089CFC0CF6C2F70E090E080E0982F872FCB
:1046D000762F6627610F711D811D911DDF91CF918E
:1046E0001F91FF90EF90DF90CF90BF90AF909F9081
:1046F0008F9008950E94D433FB0101900020E9F7C8
:104700003197AF01461B570BDC01ED91FC91028004
:10471000F381E02D09948F929F92AF92BF92EF9216
:10472000FF920F931F93CF93DF93CDB7DEB7A1977F
:104730000FB6F894DEBF0FBECDBF7C01FA01CB01EE
:1047400019A2223008F42AE08E010F5D1F4F822E3D
:10475000912CB12CA12CBF01A50194010E9498338A
:10476000F901CA016A300CF5605DD8016E938D01C4
:10477000232B242B252B79F790E080E0109721F054
:10478000BD01C7010E947C23A1960FB6F894DEBF3D
:104790000FBECDBFDF91CF911F910F91FF90EF9092
:1047A000BF90AF909F908F900895695CDECF462FA9
:1047B00050E070E060E02AE00C948B238F929F928F
:1047C000AF92BF92CF92DF92EF92FF920F931F931F
:1047D000CF93DF93FC01268527FD92C08B01EC016E
:1047E00061E070E080E090E00E94C9130E94A41391
:1047F0006B017C012E8530E0F901E255FA4F84917E
:10480000F901E656FA4FB490F901EA57FA4FA4902D
:10481000AA2009F472C081110E941113EA2DF0E060
:10482000EE0FFF1FE859FF4FA591B491EC91BE2206
:1048300031E020E009F430E0832F922F2F85022E03
:10484000000C330B2817390711F561E070E080E0A8
:1048500090E00E94C9130E94A4136C197D098E096F
:104860009F0988889988AA88BB8886169706A80613
:10487000B90608F0BFCF69E971E08CEC92E00E94C4
:104880007C2367EA71E08CEC92E00E947C230115A6
:10489000110509F446C08C89882309F442C00E949E
:1048A000A4139B01AC012C193D094E095F09690154
:1048B0007A01B8018CEC92E00E947C236AEA71E0F4
:1048C0008CEC92E00E947C232AE0B701A6018CECDC
:1048D00092E00E948B2367EA71E08CEC92E0DF911A
:1048E000CF911F910F91FF90EF90DF90CF90BF90ED
:1048F000AF909F908F900C947C2390E080E09ECFAF
:10490000BA0190E080E0DF91CF911F910F91FF906D
:10491000EF90DF90CF90BF90AF909F908F900C94CE
:10492000C913DF91CF911F910F91FF90EF90DF900E
:10493000CF90BF90AF909F908F900895CF93DF93CB
:10494000EC018A8D882399F062E2CE010E94EB206F
:1049500063E8CE010E94CC2060E2CE010E94EB20F1
:1049600046E950E06EEA71E0CE010E94DE231A8E25
:104970001B8EDF91CF9108950C949E24CF93DF93EB
:10498000EC010E949E248D8587FD0AC060E1CE0166
:104990000E94EB2061E0CE010E94CC2081E08C8F50
:1049A000DF91CF910895CF93DF93EC018A8D811130
:1049B00013C062E2CE010E94EB2068EFCE010E949C
:1049C000CC2060E2CE010E94EB2044E650E068EB90
:1049D00071E0CE010E94DE2381E08A8FDF91CF91CA
:1049E0000895CF93DF93EC010E948221CE010E94B3
:1049F000D32481E08B8FDF91CF9108952F923F9246
:104A00004F925F926F927F928F929F92AF92BF92DE
:104A1000CF92DF92EF92FF920F931F93CF93DF938A
:104A2000CDB7DEB72E970FB6F894DEBF0FBECDBF61
:104A30003C0169875B874A8719012801FA82E9826C
:104A40000BA11CA1EDA0FEA02FA12C8738A53D87AE
:104A500089A58E87D30158968C915897882341F069
:104A6000ED91FC910680F781E02D6FEFC301099570
:104A700061E070E080E090E00E94C913E981FA8172
:104A8000F7FD1AC1D7FC18C117FD16C1F7FC14C1F8
:104A900037FC12C12E163F060CF00EC157FC0CC19C
:104AA0004C145D040CF008C1960124193509E21676
:104AB000F3060CF49701C50168E070E00E948433AE
:104AC000A501481B590BC101887F69817A81681B48
:104AD000790B061717070CF4B8015B01F7E0AF0E6E
:104AE000B11CB7FE04C05B018EE0A80EB11C98EFAC
:104AF000A9227A0157FF02C0F12CE12CBA016A0DFC
:104B00007B1D683C71052CF088EC90E05C01A41AD8
:104B1000B50AB401620F731F683C710524F028ECDC
:104B200030E028193909D701A41BB50BB887AF832A
:104B3000AA1ABB0A1A141B040CF0BEC09C828B82FA
:104B400097FE02C01C821B82EB81FC81E819F909E7
:104B50004F01C9018E1B9F0B9E838D83181619066A
:104B60000CF0AAC0D3015B968C91811103C0C301E4
:104B70000E94F1240D811E8195014B815C81B7015A
:104B8000C3010E9416216985C3010E94EB20F50133
:104B900043E0F595E7954A95E1F7FC83EB835101F6
:104BA00053E0B594A7945A95E1F78F81988597FDC6
:104BB000079623E0959587952A95E1F7E980FA8095
:104BC000F7E0EF0EF11C33E0F594E7943A95E1F746
:104BD00010E000E01401240C351C9601241935095D
:104BE00029014818590831E0431A5108A80EB91E86
:104BF000C101800F911F8E9D90018F9D300D9E9D54
:104C0000300D1124C201801B910B8E9D40018F9DA0
:104C1000900C9E9D900C1124D12CC12CC501820FAB
:104C2000931F9A8389838A0C9B1CAB81BC81AC1532
:104C3000BD05E1F0BD85F401B11102C0E981FA8141
:104C4000EC0DFD1D2A853B85E20FF31F3E853323C6
:104C500059F064918C8581116095C3010E94CC202C
:104C60009FEFC91AD90AE1CF6081F4CF0F5F1F4FC0
:104C7000AD81BE81A017B10709F0BACF61E070E045
:104C800080E090E02E960FB6F894DEBF0FBECDBF49
:104C9000DF91CF911F910F91FF90EF90DF90CF9018
:104CA000BF90AF909F908F907F906F905F904F904C
:104CB0003F902F900C94C9132E960FB6F894DEBF38
:104CC0000FBECDBFDF91CF911F910F91FF90EF905D
:104CD000DF90CF90BF90AF909F908F907F906F901C
:104CE0005F904F903F902F9008958F929F92AF9238
:104CF000BF92CF92DF92EF92FF920F931F93CF93C9
:104D0000DF93CDB7DEB7EF85F889AB89AF93AA897A
:104D1000AF93A989AF93FF93EF939F928F92450131
:104D200056016701780189019A01AB0166E20E9490
:104D3000FE240FB6F894DEBF0FBECDBFDF91CF913A
:104D40001F910F91FF90EF90DF90CF90BF90AF90A9
:104D50009F908F9008958F929F92AF92BF92CF9223
:104D6000DF92EF92FF920F931F93CF93DF93CDB714
:104D7000DEB7EF85F889AB89AF93AA89AF93A9898C
:104D8000AF93FF93EF939F928F9245015601670176
:104D9000780189019A01AB0164E20E94FE240FB6FA
:104DA000F894DEBF0FBECDBFDF91CF911F910F9161
:104DB000FF90EF90DF90CF90BF90AF909F908F903B
:104DC00008952F923F924F925F926F927F928F92AF
:104DD0009F92AF92BF92CF92DF92EF92FF920F938A
:104DE0001F93CF93DF93CDB7DEB72A970FB6F89412
:104DF000DEBF0FBECDBF3C016D835F834E832901B3
:104E0000A88689862F8D2A87DC0158968C91589721
:104E1000882341F0ED91FC910680F781E02D6FEF42
:104E2000C301099561E070E080E090E00E94C91341
:104E3000C701079697FD07967C0153E0F594E79428
:104E40005A95E1F7C20168E070E00E948433F201F4
:104E5000E81BF90BCF01270163E0440C551C6A9550
:104E6000E1F75F01F7FF02C0B12CA12C9C01240DDA
:104E7000351D283C31052CF048EC442E512C481AA5
:104E8000590A98012C0D3D1D283C31050CF479C0C0
:104E900028EC30E0201B310BA501481B590B5C832B
:104EA0004B83441A550A141415040CF09CC0480195
:104EB00017FF02C0912C812C1401201A310AC9015C
:104EC000821993099A838983181619060CF08BC0EE
:104ED000D3015B968C91811103C0C3010E94F12420
:104EE00009811A819201A401B501C3010E94162112
:104EF0006D81C3010E94EB20820133E01595079577
:104F00003A95E1F78B819C8197FD079623E0959573
:104F100087952A95E1F7B1E0CB1AD108C218D308DA
:104F2000CE9C5001CF9CB00CDE9CB00C1124A80E7E
:104F3000B91E2E9C60012F9CD00C3E9CD00C1124DD
:104F4000C80ED91E512C412C912C812C0815190505
:104F500001F1E985EE23B9F0F401EA0DFB1D2E8184
:104F60003F81E20FF31F3A85332389F0649148852E
:104F700041116095C3010E94CC205FEF851A950A0C
:104F8000E5CF960189CFF401EC0DFD1DE8CF6081DE
:104F9000EECF8FEF481A580AAE18BF08CE0CDF1CB0
:104FA000A981BA81A415B50579F661E070E080E0C9
:104FB00090E02A960FB6F894DEBF0FBECDBFDF910A
:104FC000CF911F910F91FF90EF90DF90CF90BF9006
:104FD000AF909F908F907F906F905F904F903F9099
:104FE0002F900C94C9132A960FB6F894DEBF0FBE0B
:104FF000CDBFDF91CF911F910F91FF90EF90DF9088
:10500000CF90BF90AF909F908F907F906F905F9068
:105010004F903F902F9008958F92AF92CF92DF9252
:10502000EF92FF920F931F93CF93DF93CDB7DEB72D
:105030008F928A2CAC2C6701780189019A01AB010F
:1050400066E20E94E1260F90DF91CF911F910F91B0
:10505000FF90EF90DF90CF90AF908F9008958F9258
:10506000AF92CF92DF92EF92FF920F931F93CF9365
:10507000DF93CDB7DEB78F928A2CAC2C6701780115
:1050800089019A01AB0164E20E94E1260F90DF9151
:10509000CF911F910F91FF90EF90DF90CF90AF9045
:1050A0008F9008951F93CF93DF93EC01162F8B8D74
:1050B000811103C0CE010E94F124412F66E2CE018E
:1050C000DF91CF911F910C94F9211F93CF93DF9320
:1050D000EC01162F188E8B8D811103C0CE010E941A
:1050E000F124412F64E2CE010E94F921898D8823A9
:1050F00041F0412F66E2CE01DF91CF911F910C94D8
:10510000F921DF91CF911F9108958F929F92AF92D5
:10511000BF92CF92DF92EF92FF920F931F93CF93A4
:10512000DF93EC01FB014A01898D8823A1F0E8811E
:10513000F9810288F389E02D60E0CE01DF91CF9103
:105140001F910F91FF90EF90DF90CF90BF90AF90A5
:105150009F908F90099498E0C92ED12CCB01B60175
:105160000E948433E81BF90BCF01B6010E948433FF
:105170007901E81AF90A6F01F7FF02C0D12CC12C9E
:10518000540197FE02C0B12CA12CCF018E0D9F1DA2
:10519000883C91052CF088ECE82EF12CEE1AFF0AE1
:1051A000C401800F911F883C910524F008EC10E0A9
:1051B00008191909C6018E1B9F0BE81AF90AC501C7
:1051C00088199909081B190B8B8D811103C0CE0119
:1051D0000E94F1249701A501B601CE010E9416217B
:1051E00062E2CE010E94EB206CEFCE010E94CC2047
:1051F00060E2CE010E94EB2044EF51E061EC71E0EF
:10520000CE01DF91CF911F910F91FF90EF90DF9032
:10521000CF90BF90AF909F908F900C94DE230F9310
:105220001F93CF93DF93EC01662399F0E881F98116
:105230000488F589E02D08EC10E028EC30E050E01F
:1052400040E070E060E00995DF91CF911F910F91F0
:1052500008958B8D882339F0CE010E948221CE01E2
:105260000E94D3241B8E62E2CE010E94EB2064EFE9
:10527000CE010E94CC2060E2CE010E94EB2048E2E9
:105280005AE06EEC71E0CE010E94DE23198EDCCF75
:1052900085ED8093BC008091A4029091A502A0911D
:1052A000A602B091A7020796A11DB11D23E0B695F5
:1052B000A795979587952A95D1F72091BC0024FD55
:1052C00003C01092A20208954091A4025091A50239
:1052D0006091A6027091A702452B462B472B69F3DC
:1052E0000097A105B10541F025E32A95F1F70000EB
:1052F0000197A109B109E1CF8091A3020C94C71BCA
:1053000060E071E088EF91E00E94D93340E168EFFE
:1053100071E087E00E944D2261E085E00E943A132F
:1053200061E070E080E090E00E94C91360E085E0F9
:105330000E943A1360E08FEF0E94132285FFFACF9C
:1053400060E287E00C9413221F920F920FB60F9227
:1053500011242F933F934F935F936F937F938F937A
:105360009F93AF93BF93EF93FF938CEC92E00E94D7
:105370008212FF91EF91BF91AF919F918F917F9199
:105380006F915F914F913F912F910F900FBE0F90B2
:105390001F9018951F920F920FB60F9211242F9302
:1053A0008F939F93EF93FF93E091DC02F091DD02E6
:1053B0008081E091E202F091E30282FD1BC09081C6
:1053C0008091E5028F5F8F732091E602821741F092
:1053D000E091E502F0E0E453FD4F958F8093E50204
:1053E000FF91EF919F918F912F910F900FBE0F9092
:1053F0001F9018958081F4CF1F920F920FB60F92D5
:1054000011242F933F938F939F93AF93BF938091DA
:105410004E0290914F02A0915002B09151023091F2
:105420004D0223E0230F2D3758F50196A11DB11D24
:1054300020934D0280934E0290934F02A09350020E
:10544000B09351028091520290915302A091540264
:10545000B09155020196A11DB11D80935202909307
:105460005302A0935402B0935502BF91AF919F9104
:105470008F913F912F910F900FBE0F901F90189515
:1054800026E8230F0296A11DB11DD2CF1F920F92C5
:105490000FB60F9211242F933F934F935F936F9307
:1054A0007F938F939F93AF93BF93EF93FF938091DD
:1054B000B900887F803609F44AC0F0F5883209F4D3
:1054C000A7C018F5803109F49BC0B8F4882309F40B
:1054D000F9C0883009F494C0FF91EF91BF91AF916A
:1054E0009F918F917F916F915F914F913F912F91FC
:1054F0000F900FBE0F901F901895883109F488C047
:10550000803251F78093A00214C0803409F49DC00A
:1055100040F48033B9F38833F9F68093A00285EC28
:10552000B0C0803509F485C0883509F496C0883448
:1055300099F60E944829D0CF883909F48CC038F5F3
:10554000883729F050F4883611F0803729F683E047
:105550008093A20210924C0257C0883809F47BC095
:10556000803919F0803809F0B7CF80914C02803231
:1055700008F071C0E0914C0281E08E0F80934C02E4
:105580008091BB00F0E0E45DFD4F80833DC0803B37
:1055900039F0E0F4803A09F479C0883A09F09CCFF8
:1055A00084E08093A20210922B0210922A02E091D2
:1055B0005802F0915902099580912A0281110FC079
:1055C00081E080932A0210920A0209C0803C09F40B
:1055D000A6CF883C09F4A3CF883B09F07DCFE091AA
:1055E0002B0281E08E0F80932B02F0E0E65FFD4FEF
:1055F00080818093BB0090912B0280912A0229C068
:1056000080917D028093BB0085EC8093BC0064CFC9
:1056100090919F0280919E02981758F5E0919F0209
:1056200081E08E0F80939F02F0E0E258FD4F808171
:10563000E9CFE0919F0281E08E0F80939F028091DD
:10564000BB00F0E0E258FD4F808390919F02809173
:105650009E029817C8F285E8D8CFE0919F0281E0BA
:105660008E0F80939F028091BB00F0E0E258FD4FC7
:1056700080838091A10281115CCF81E080937C02C4
:1056800084EA8093BC001092A20226CF85EC80931E
:10569000BC001092A20280914C02803230F4E09162
:1056A0004C02F0E0E45DFD4F108260914C0270E02E
:1056B000E0915602F09157028CE292E00995109227
:1056C0004C020ACF1092A00234CFCF92DF92EF9219
:1056D000FF92ECECF2E01382128288EE93E0A0E0FD
:1056E000B0E084839583A683B78321E231E03183E0
:1056F000208325EC30E03587248724EC30E03787A1
:10570000268720EC30E0318B208B21EC30E0338B8E
:10571000228B22EC30E0358B248B26EC30E0378B6B
:10572000268B118E128E138E148EE9E6F3E013820F
:10573000128284839583A683B78383E391E0918368
:105740008083EDEAF3E01382128228EC30E03583A7
:105750002483378326833187208733872287168ADD
:10576000158614861786168681E0858B848B4FEF0D
:105770005FEF538B428B518B408B878B108E128E39
:10578000118E41E551E051834083368F258F30A340
:10579000278F41E050E052A341A313A284A385A325
:1057A0009AE096A399E097A398E090A797E091A735
:1057B00082A790E8C92E96E9D92E98E9E92EF12C16
:1057C000C3A6D4A6E5A6F6A617A610AA90E591ABA7
:1057D00012AA83AB84AB15AA16AA17AA64E170E0DB
:1057E00071AF60AF6DE771E0748F638F60E270E05E
:1057F000709314076093130767E070E070931207CB
:105800006093110710920A07109209071092070778
:105810001092100710920F0710921607109215079A
:10582000109218071092170730931A072093190740
:1058300030931C0720931B07E5E7F3E013821282E5
:1058400025E431E03183208317821682578746870B
:10585000878B108E12AA11AA14AA13AA17AAFF9056
:10586000EF90DF90CF900895CF93DF9300D000D0DA
:105870001F92CDB7DEB7789484B5826084BD84B5BD
:10588000816084BD85B5826085BD85B5816085BD3B
:1058900080916E00816080936E00109281008091F3
:1058A000810082608093810080918100816080937B
:1058B0008100809180008160809380008091B100A0
:1058C00084608093B1008091B00081608093B000CB
:1058D00080917A00846080937A0080917A0082605F
:1058E00080937A0080917A00816080937A00809121
:1058F0007A00806880937A001092C10010925B0257
:1059000010925A021092C9021092C8020E94A91B5A
:1059100082E092E1909359028093580283E092E1F1
:1059200090935702809356020E94481D61E086E0E2
:105930000E94681361E086E00E943A1361E085E00E
:105940000E94681360E085E00E943A1385E0E8E178
:10595000F1E0DE01119601900D928A95E1F768EC75
:1059600070E080E090E00E94C91360E787E00E9449
:10597000132260E082E00E94132260E081E00E9436
:10598000132260E181E10E94132280E00E9439220B
:10599000682F6C6080E00E94132263E083E00E9425
:1059A000132240E0BE016F5F7F4F86E00E944D22D0
:1059B00080E00E943922682F6E7F80E00E941322CF
:1059C00064E685E00E94132280E00E943922682F5D
:1059D000626080E00E94132262E070E080E090E06C
:1059E0000E94C91340E050E0BA0188EC93E00E94A5
:1059F0006C1B109207071092100710920F0710925D
:105A00001607109215071092180710921707809129
:105A1000B1039091B20390931A0780931907809174
:105A2000B3039091B40390931C0780931B078DEAF6
:105A300093E090937A03809379038EE480937C00C3
:105A400020E031E080E090E0DC0140917A00406CA1
:105A500040937A0040917A0046FDFCCF4091780057
:105A600050917900840F951FA11DB11D215031095E
:105A700061F720917A002F7720937A00BC01CD0145
:105A8000E4E09595879577956795EA95D1F7072E88
:105A9000000C880B990B0E9416319B01AC0161E64A
:105AA00073E583ED99E40E94D7320E944933CB011C
:105AB00064E670E00E9484336093170180931601BE
:105AC00064E670E080E090E00E94C9136AE070E054
:105AD00080E090E00E94C91383EE90E00E94661C73
:105AE0000E9489220E94163120E030E040E857E30E
:105AF0000E94753122E538EB4FE253E40E94753184
:105B000026E636E64BE352E40E946A322DEC3CEC8A
:105B10004CE85FE30E946A322B013C0164E670E0CE
:105B200080E090E00E94C91385EE90E00E94661C20
:105B30000E9489220E94163120E030E040E857E3BD
:105B40000E94753120E030E04AEF52E40E94753146
:105B500020E030E040EC50E40E946A326B017C01AE
:105B6000C301B2010E945033162F6093150120E04B
:105B700030E040E251E4C301B2010E9475312B01D3
:105B80003C012AE0129FB0011124072E000C880B63
:105B9000990B0E9416319B01AC01C301B2010E9416
:105BA0006A322B013C0120E030E0A9010E947F33E2
:105BB00018160CF01EC2C301B2010E94503360934C
:105BC0001401C701B6010E945033162F60931301D0
:105BD00020E030E040E251E4C701B6010E94753197
:105BE0006B017C013AE0139FB0011124072E000CD9
:105BF000880B990B0E9416319B01AC01C701B601BD
:105C00000E946A320E9450336093120161E08DEA73
:105C100093E00E947A1510920707109216071092CF
:105C2000150710921807109217078091B1039091F1
:105C3000B20390931A07809319078091B303909150
:105C4000B40390931C0780931B0781E080938C031F
:105C500010928D0310928403109283038FEF9FEFB5
:105C600090938603809385036FEF7FEF8DEA93E037
:105C70000E94E01E1092100710920F071092080762
:105C800042E3642E712C59E6452E512C64E6962E83
:105C900075E0272E312CDD24D3946FEF7FEF8DEA52
:105CA00093E00E94E01EB12CA12CC12CF12CE12C20
:105CB00010E000E0C80187709927CC0C892B59F4BB
:105CC000F80133E0F595E7953A95E1F7EA0DFB1D0C
:105CD000EE53FA4FC490C7FC08C030E020E0A701A3
:105CE000B8018DEA93E00E94251E0F5F1F4F083C0C
:105CF000110501F74FEFE41AF40A89E1A80EB11C6F
:105D000098ECE916F104A1F68BE29FE10E94FA14E7
:105D10007092BA036092B9037092BC036092BB03A5
:105D20007092A7036092A6035092A9034092A80321
:105D30001092AC036091150185E793E00E94D72390
:105D40006BED71E085E793E00E947C238EE89CE197
:105D50000E94FA1421E930E03093A7032093A603B0
:105D60005092A9034092A8031092AC0360911401D1
:105D700085E793E00E94D7238CE390E09093A703FC
:105D80008093A60324EB30E03093A9032093A8036B
:105D90001092AC036091130185E793E00E94D72332
:105DA0006BED71E085E793E00E947C236091120126
:105DB00085E793E00E94D7238AE499E10E94FA14D0
:105DC0008BE490E09093A7038093A6032FE030E04C
:105DD0003093A9032093A8031092AC03609117019C
:105DE00085E793E00E94D7236BED71E085E793E0B0
:105DF0000E947C23609116016A3040F46DED71E0E1
:105E000085E793E00E947C236091160185E793E08B
:105E10000E94D723209117018091160190E0299DBF
:105E2000800D911D1124883131E0930714F488E12D
:105E300091E088519140B1010E9484336E5F6C31D2
:105E400008F06BE1262F30E0F12CE12C01E110E0AD
:105E500046E050E062E170E08DEA93E00E947A193A
:105E60004091110750911207E09107074130510509
:105E700009F0F8C0EE2309F4C4C0E0901B07F090CD
:105E80001C070091190710911A0780910A078823AF
:105E900009F4B3C02091B3033091B4032E193F0924
:105EA000209FC001219F900D309F900D112423E071
:105EB000969587952A95E1F79C0129513C4F390128
:105EC0002091170730911807409115075091160738
:105ED000812CA12CC12CB30188EC93E00E942F28C7
:105EE00000911B0710911C072091190730911A0788
:105EF0004091170750911807609115077091160788
:105F000088EC93E00E948528E0901B07F0901C0726
:105F10000091190710911A0720911707309118075F
:105F20004091150750911607B30188EC93E00E9449
:105F30000C2860ED77E080E090E00E94C91388ECC7
:105F400093E00E949E241F9288E38F933091130167
:105F50002AE08091120190E0329F800D911D112462
:105F60009F938F93309117018091160190E044E642
:105F7000349F800D911D11249F938F9330911501B3
:105F80008091140190E0329F800D911D11249F9308
:105F90008F938FED91E09F938F9380E091E09F939B
:105FA0008F930E94E0330E94802968EE73E080E0C6
:105FB00090E00E94C9130E94802983B7817F84608A
:105FC00083BF83B7816083BF889583B78E7F83BF8C
:105FD0000FB6F894DEBF0FBECDBF00E010E0011594
:105FE0001105E9F30E946E128823C9F30E94000094
:105FF000F6CFC301B2019058E0CD80E090E0DC0123
:106000005BCFE090B303F090B4030091B103109123
:10601000B203812CA12CC12C30E020E050E040E004
:1060200067EE73E088EC93E00E942F2860E088EC34
:1060300093E00E940F29E090B303F090B403009125
:10604000B1031091B20330E020E050E040E067EE91
:1060500073E088EC93E00E940C2888EC93E00E94A7
:106060009E2467CF60910F077091100780911307EE
:1060700090911407689F9001699F300D789F300DB3
:106080001124EE2309F48FC041505109641775079C
:1060900008F07BC0AC01420F531FE0901707F0904F
:1060A00018072E0D3F1D60911B0770911C074E0DA8
:1060B0005F1DE60EF71E4E155F0508F47A012E15DA
:1060C0003F0570F50091190710911A0740910A07D2
:1060D000442309F45FC0820F931F8E199F09809F8C
:1060E000B001819F700D909F700D112483E0769513
:1060F00067958A95E1F7CB01E21AF30A40911507FB
:1061000050911607BC0169517C4F80910807812C82
:10611000A12CC12C811142C088EC93E00E942F2851
:1061200080910F079091100701969093100780932C
:106130000F07209111073091120782179307F1F48E
:106140001092100710920F07809108078111F1CE6D
:1061500000911B0710911C072091190730911A0715
:106160004091170750911807609115077091160715
:1061700088EC93E00E948528D09208076FEF7FEFAC
:106180008DEA93E00E94E01E88CD4091B3035091C8
:10619000B40383CF80E090E0DC01AECF88EC93E0E5
:1061A0000E940C28BDCFE090B303F090B403E21A34
:1061B000F30A8E159F0508F47C010091B10310913C
:1061C000B20380910807812CA12CC12C50E040E043
:1061D00067EE73E0811123C088EC93E00E942F28C2
:1061E00080910F079091100701969093100780936C
:1061F0000F0720911107309112078217930709F0BA
:10620000BDCF1092100710920F07809108078111DF
:1062100024CF60E088EC93E00E940F29ADCF88EC9A
:1062200093E00E940C28DCCFE89409C097FB3EF471
:1062300090958095709561957F4F8F4F9F4F9923D3
:10624000A9F0F92F96E9BB279395F6958795779551
:106250006795B795F111F8CFFAF4BB0F11F460FF11
:106260001BC06F5F7F4F8F4F9F4F16C0882311F069
:1062700096E911C0772321F09EE8872F762F05C07D
:10628000662371F096E8862F70E060E02AF09A9518
:10629000660F771F881FDAF7880F9695879597F90D
:1062A0000895990F0008550FAA0BE0E8FEEF1616A7
:1062B0001706E807F907C0F012161306E407F507FA
:1062C00098F0621B730B840B950B39F40A2661F06E
:1062D000232B242B252B21F408950A2609F4A14011
:1062E000A6958FEF811D811D08950E9488310C9421
:1062F000F9310E94EB3138F00E94F23120F0952301
:1063000011F00C94E2310C94E83111240C942D32EC
:106310000E940A3270F3959FC1F3950F50E0551F0C
:10632000629FF001729FBB27F00DB11D639FAA27EA
:10633000F00DB11DAA1F649F6627B00DA11D661F39
:10634000829F2227B00DA11D621F739FB00DA11D5A
:10635000621F839FA00D611D221F749F3327A00D14
:10636000611D231F849F600D211D822F762F6A2FB0
:1063700011249F5750409AF0F1F088234AF0EE0F15
:10638000FF1FBB1F661F771F881F91505040A9F742
:106390009E3F510580F00C94E2310C942D325F3F0A
:1063A000E4F3983ED4F3869577956795B795F7957E
:1063B000E7959F5FC1F7FE2B880F911D96958795F6
:1063C00097F9089597F99F6780E870E060E0089575
:1063D0009FEF80EC089500240A94161617061806FD
:1063E0000906089500240A941216130614060506D9
:1063F0000895092E0394000C11F4882352F0BB0F6A
:1064000040F4BF2B11F460FF04C06F5F7F4F8F4FCC
:106410009F4F089557FD9058440F551F59F05F3F07
:1064200071F04795880F97FB991F61F09F3F79F0B6
:1064300087950895121613061406551FF2CF469538
:10644000F1DF08C0161617061806991FF1CF8695BA
:106450007105610508940895E894BB27662777279E
:10646000CB0197F908952F923F924F925F926F92CE
:106470007F928F929F92AF92BF92CF92DF92EF92D4
:10648000FF920F931F93CF93DF93CDB7DEB7CA1B55
:10649000DB0B0FB6F894DEBF0FBECDBF09942A8880
:1064A000398848885F846E847D848C849B84AA8428
:1064B000B984C884DF80EE80FD800C811B81AA81B5
:1064C000B981CE0FD11D0FB6F894DEBF0FBECDBF80
:1064D000ED0108955058BB27AA270E9482320C94E0
:1064E000F9310E94EB3138F00E94F23120F039F49A
:1064F0009F3F19F426F40C94E8310EF4E095E7FB85
:106500000C94E231E92F0E940A3258F3BA1762075D
:1065100073078407950720F079F4A6F50C942C32C4
:106520000EF4E0950B2EBA2FA02D0B01B9019001AE
:106530000C01CA01A0011124FF27591B99F0593FF2
:1065400050F4503E68F11A16F040A22F232F342F3A
:106550004427585FF3CF469537952795A795F04088
:106560005395C9F77EF41F16BA0B620B730B840B9D
:10657000BAF09150A1F0FF0FBB1F661F771F881F55
:10658000C2F70EC0BA0F621F731F841F48F48795AD
:1065900077956795B795F7959E3F08F0B0CF93959F
:1065A000880F08F09927EE0F9795879508950E9418
:1065B000EB320C94F9310E94F23158F00E94EB3129
:1065C00040F029F45F3F29F00C94E23151110C9412
:1065D0002D320C94E8310E940A3268F39923B1F30A
:1065E000552391F3951B550BBB27AA2762177307F9
:1065F000840738F09F5F5F4F220F331F441FAA1F8D
:10660000A9F335D00E2E3AF0E0E832D09150504048
:10661000E695001CCAF72BD0FE2F29D0660F771FF6
:10662000881FBB1F261737074807AB07B0E809F0DC
:10663000BB0B802DBF01FF2793585F4F3AF09E3F61
:10664000510578F00C94E2310C942D325F3FE4F365
:10665000983ED4F3869577956795B795F7959F5FA4
:10666000C9F7880F911D9695879597F90895E1E0F0
:10667000660F771F881FBB1F621773078407BA074F
:1066800020F0621B730B840BBA0BEE1F88F7E095AA
:1066900008950E9450336894B1110C942D320895DE
:1066A0000E94123288F09F5798F0B92F9927B7515E
:1066B000B0F0E1F0660F771F881F991F1AF0BA95A6
:1066C000C9F714C0B13091F00E942C32B1E00895A6
:1066D0000C942C32672F782F8827B85F39F0B93F98
:1066E000CCF3869577956795B395D9F73EF4909559
:1066F0008095709561957F4F8F4F9F4F08950E94B1
:10670000513108F48FEF089597FB072E16F400948B
:1067100007D077FD09D00E94BA3307FC05D03EF4BC
:10672000909581959F4F0895709561957F4F08953D
:10673000A1E21A2EAA1BBB1BFD010DC0AA1FBB1F85
:10674000EE1FFF1FA217B307E407F50720F0A21BF7
:10675000B30BE40BF50B661F771F881F991F1A9464
:1067600069F760957095809590959B01AC01BD018E
:10677000CF010895AA1BBB1B51E107C0AA1FBB1F75
:10678000A617B70710F0A61BB70B881F991F5A95BD
:10679000A9F780959095BC01CD010895EE0FFF1FDC
:1067A0000590F491E02D099481E090E0F8940C9428
:1067B0008136FB01DC0101900D920020E1F7089584
:1067C000AEE0B0E0E6EEF3E30C9441320D891E89B1
:1067D00086E08C831A8309838FEF9FE79E838D83E6
:1067E000AE01475E5F4F6F89788DCE0101960E94A2
:1067F00003342F813885020F131FF80110822E9663
:10680000E4E00C945D32ABE0B0E0E9E0F4E30C943A
:1068100033327C013B018A01FC011782168283819D
:1068200081FFC8C1CE0101965C01F7019381F3019C
:1068300093FD859193FF81913F01882309F453C112
:10684000853239F493FD859193FF81913F01853223
:1068500029F4B70190E00E94F335E7CF912C212C69
:10686000312CFFE1F31538F08B3211F190F48032C6
:1068700009F1833229F137FC3CC020ED280F2A3082
:1068800050F536FE20C08AE0989E200D1124922EED
:1068900006C08D3291F0803371F7689430F8F301BF
:1068A00093FD859193FF81913F018111DACF21C042
:1068B000689431F8689432F8F2CF689433F8EFCFE7
:1068C000689434F8ECCFEAE02E9E200D1124222E9D
:1068D000689435F8E4CF8E3229F436FC04C168940C
:1068E00036F8DDCF8C3619F4689437F8D8CF88366F
:1068F000B1F2982F9F7D95549330E0F08336A1F14B
:106900008337C1F1833509F063C02801F2E04F0EEF
:10691000511CF801C080D180692D70E036FC02C0A6
:106920006FEF7FEFC6010E94DD354C01689437F8A8
:1069300082010AC00C5F1F4FFFE3F9838824839410
:10694000912C6501E89437F833FE2DC0522C811448
:10695000910471F5552009F468CFB70180E290E009
:106960000E94F3355A94F6CFF801808189830E5F37
:106970001F4FE4CF2801F2E04F0E511CF801C080F8
:10698000D180692D70E036FC02C06FEF7FEFC60149
:106990000E94E8354C018201D5CFB70180E290E03A
:1069A0000E94F3352A942814190409F0B0F7CECFC9
:1069B000F60137FC859137FE81916F01B70190E0B8
:1069C0000E94F33551105A94F1E08F1A9108BFCF0D
:1069D000843619F0893609F077C0F80137FE6BC0AC
:1069E00060817181828193810C5F1F4FF32DFF764F
:1069F0003F2E97FF09C090958095709561957F4FC8
:106A00008F4F9F4F689437F82AE030E0A5010E942D
:106A10002336C82ECA188C2C432C36FE0CC0E894A2
:106A200040F8C91440F434FE05C032FC03C0F32D15
:106A3000FE7E4F2E892C44FE95C0FE01EC0DF11D0B
:106A40008081803309F087C0242D297E422E842D39
:106A50008870582E43FC95C040FE8FC09C2C821439
:106A600018F42C0C922C981844FE91C0B70180E3C6
:106A700090E00E94F33542FE09C088E790E041FEB5
:106A800002C088E590E0B7010E94F335C91408F40C
:106A90008AC0CA94D12C9FEFC91AD90ACA0CDB1C30
:106AA000F60182916F01B70190E00E94F335AC14BA
:106AB000BD04B1F74FCF60817181072E000C880BA8
:106AC000990B0E5F1F4F92CFD32CE894D4F82AE095
:106AD00030E0853739F1232D297FD22E8F3601F111
:106AE00048F48835A9F0F701868197812B96E2E179
:106AF0000C944F32803749F08837A9F7D4FE02C092
:106B00006894D2F820E130E00DC06894D4F8F6CF54
:106B100034FE03C0822F8660D82E20E132E002C00E
:106B200028E030E0F801D7FE0FC0608171818281DA
:106B300093810C5F1F4FA5010E942336C82ECA18EF
:106B40003D2CE89437F867CF6081718190E080E058
:106B50000E5F1F4FF0CF42FC02C0839478CF839426
:106B6000839475CF842D867809F471CFF6CFB70161
:106B700080E290E00E94F33583948214C0F3512C9C
:106B800073CF522C5818821408F46ECFF8CF842D8E
:106B9000867809F47BCF8BE241FE80E247FC8DE2F0
:106BA000B70190E071CFB70180E390E00E94F33528
:106BB0009A946CCF8FEF9FEF99CFFC0105906150B5
:106BC00070400110D8F7809590958E0F9F1F089503
:106BD000FC016150704001900110D8F780959095AC
:106BE0008E0F9F1F08950F931F93CF93DF93182F3E
:106BF000092FEB018B8181FD09C01FEF0FEF812F62
:106C0000902FDF91CF911F910F91089582FF14C0B3
:106C10002E813F818C819D81281739073CF4E881C2
:106C2000F981CF0101969983888310838E819F819A
:106C300001969F838E83E3CFE885F985812F09959F
:106C4000892BA1F3DACFFA01AA27283051F120319C
:106C500081F1E8946F936E7F6E5F7F4F8F4F9F4FF0
:106C6000AF4FB1E03ED0B4E03CD0670F781F891F32
:106C70009A1FA11D680F791F8A1F911DA11D6A0F00
:106C8000711D811D911DA11D20D009F468943F91B3
:106C90002AE0269F11243019305D3193DEF6CF01B2
:106CA0000895462F4770405D4193B3E00FD0C9F778
:106CB000F6CF462F4F70405D4A3318F0495D31FDE5
:106CC0004052419302D0A9F7EACFB4E0A695979538
:106CD000879577956795BA95C9F70097610571050E
:106CE00008959B01AC010A2E069457954795379558
:106CF0002795BA95C9F7620F731F841F951FA01DB2
:066D00000895F894FFCF96
:106D060074312B333333633333763239396839355B
:106D16007300064B03191403E2E423E402000000A7
:106D260000A41204123112F112621240125412001F
:106D3600000000371C0A1C8622311AFB11F71BE8DB
:106D46001B00000000161FEE1E86226B20000000AE
:106D560000B417041286226B20251E311A5A1A32E5
:106D66001A4E1A421A611A311A7A157915F819BF8C
:106D7600197A19E01EE5188618000000006C1B7EC3
:106D86001D0E1B65282F28AB2652280C2875260FAA
:106D9600298528BC24BE246B20427573792054694A
:106DA6006D656F757421000D0A00203A20005F5052
:106DB6006F7765724F6666005F506F7765724F6ECC
:106DC600005F5570646174655F50617274005F5551
:106DD60070646174655F46756C6C002E00300074DB
:106DE600352B252E336463252E336476252E3364A6
:086DF60068252E3264730000D1
:00000001FF
